:020000040000fa
:080000000002040000000000f2
:020000040000fa
:100400006fbc2000007f2400000188000000000075
:100410000a00070011000700000020000000e000b3
:10042000020032000000020000000000423802001a
:10043000000000000040da000000fe004440a90077
:10044000001120000000e000030032000000200046
:10045000a00188004440a80000000600c0c223009c
:10046000010020001500370062004000e0804800d5
:10047000910188009001ba0062004000e0804800cd
:10048000910188009002ba0062004000e0804800bc
:100490000002eb006028e10004003a000059eb0084
:1004a0008301e900fdff3e00040037006128e10000
:1004b000010032000082eb00050007009101880076
:1004c0001001ba000200e000e7ff3a00000005005a
:1004d000910188008002780062004000e0804800be
:1004e0003559ba008301e900080032002559ba00e5
:1004f0008301e900050032000400e000f4ff32004f
:1005000015d9ba008301e900f1ff3a0000000600a6
:100510008c02040000000000881f780002047800ac
:1005200014000700080040004f0478000000060097
:100530000000fa00881f7800000478003fb9970097
:10054000ea81570080007800c028200010000700d2
:10055000800078000000e000020035000040eb0061
:1005600000f47800010078004f0478000080fa0061
:10057000000006008001eb000200370061f0790006
:100580008301e800828f5100fcff3a000000060062
:100590006200fa00889fbe008a9fbe000004be0071
:1005a000020578008300780060f92f000f004000fa
:1005b000b000070088979f0099979f000000eb000c
:1005c000a09f9f009a4578000b80fb000000ea0086
:1005d000cf04de0050c2b30080cf550002003200cd
:1005e00009047800010037000904e9000800e00070
:1005f0000b0034001f909700080178008a007800f3
:100600008f9197000300010090979f000000e00089
:10061000930032002f98970000004400a09f9f0095
:100620000905450050c2b30080cf550004003200d8
:100630000b04e000e3ff3a002f9897008900370091
:100640000000eb00809f9f00f0979f00e0979f00c5
:10065000d0979f00c0979f00b0979f00c09f9f00ba
:1006600009003700209b200000805000000040005f
:10067000619a2000e10078004f9897000100700017
:10068000c09f9f000a05e8001a4478008800fb001c
:10069000209b20007c000700800078000000e00024
:1006a000f0ff3a00a0c2b300804f54000e003a00a1
:1006b000bf8897000180e900b08f9f00100078008c
:1006c000b09f9f000000e00005003d000000ea0030
:1006d000b09f9f004f9897000020a000c09f9f00f0
:1006e0000a05e80010003700b19f9f00090037009d
:1006f000bf989700f0ff2700808f50000400320061
:100700006a08b9000000410003004000b09f9f004c
:100710000a05e8001a01fb0003fd2f000300410059
:10072000e90f5000f2ff3600e0c2b3009a4f10000c
:10073000040032000080eb00909f9f008a04780044
:100740001c0037008a04e800a0c2b300994f1000d3
:1007500007003a00bf8897000180e900b08f9f0032
:1007600010007800909f9f008a84e80011003700f5
:100770000000eb00909f9f00090037009f989700b2
:10078000f0ff2700808f5000040032006a08b90093
:100790000000410003004000909f9f008904e80092
:1007a0001901fb0003fd2f0003004100e90f500079
:1007b000f2ff3600194478008800fb00809b20007f
:1007c000310007000000e00002003a000044780019
:1007d000010037008904e800a87f9f0080c6b300ad
:1007e000804f540004003a00994f14000a003a0068
:1007f0006640500006003700c0c6b300804f54006a
:1008000005003a00994f140003003a00654040008b
:10081000a07f9f008904e8000905e800c8fb2f00bd
:100820000f04440060f92f000f0040008085e800ad
:100830008801780019417800800078000b0078006a
:100840001a0007000000e00005003a008800780068
:100850000b007800920107000000e00059ff3d0006
:100860000080eb004f05be004f04be000080fa0080
:10087000000006000200fa00f1bf9f0001087800a6
:100880000080fa0000000600040037000204e000c7
:1008900001003a00000005000000e8001041780067
:1008a000814f5100f9ff3a0000000600889fbe000a
:1008b0008a1f7800000478000102780082447800e2
:1008c0000305780070c6b300804f510021003c0042
:1008d00000c0e900804f5100de003d007240500032
:1008e000804f51004b0132000d003c006c40500025
:1008f000804f51005e013c0000c0e900804f510074
:10090000d4003d0050c2b300804f51005501320069
:100910007c404000804f510055013a00cd00370027
:1009200010c6b300804f5100ca00320004003c00e2
:1009300069405000804f51004d013a00720037006d
:1009400030c6b300804f5100180032000040e8006c
:100950000900370000c7b300804f51001e0132006c
:1009600008003c0000c0e900804f5100e400320064
:1009700065003c006540500080cf54003c013a00c7
:100980000f00370050c7b300804f51005e003200a7
:1009900063404000804f51005b00320065405000d2
:1009a000804f510032013a001a0137009180e9006e
:1009b000010a7800780090009171780032013700c8
:1009c000a8609000c0c6b30080cf50000a003a0073
:1009d0009400780064805000000a78001000be0087
:1009e0004f89de00cf91de000002be0002037800d6
:1009f000820378001300370010c7b30080cf500087
:100a000003003200a0c6b30080cf500006003a00b9
:100a10009400780068805000000a78003002be0020
:100a20002003be00070037001480e900000a7800a8
:100a30001000780000027800cfa2de0005037800e5
:100a400086037800049cbe000694be00a860900057
:100a500080c6b30080cf50000e00320020c6b30025
:100a600080cf500005003a000400fb00cf80de007c
:100a700001017800820178000a00370040c7b30006
:100a800080cf5000030032006640400080cf50000d
:100a900006003a0004007800cf80de0001017800f3
:100aa00082017800009cbe000294be003800be00a7
:100ab0002801be00e00f5000e08f5800e00f590001
:100ac000e08f590003003d0078009000d1c2b300d0
:100ad0000a003700081090000018a300030032003d
:100ae00078009000b1c2b300040037000008a300f2
:100af000530032007800900001c2b3000175780005
:100b00000000e8004d003700a8609000c0c6b300a8
:100b100080cf500006003a009400780064805000b6
:100b2000000a78001002be006033b80013003700de
:100b300010c7b30080cf500003003200a0c6b3003e
:100b400080cf500006003a00940078006880500082
:100b5000000a78003002be002003be000700370004
:100b60001480e900000a7800100078000002780084
:100b7000050020000600200007002000049cbe00a5
:100b80000694be00a860900080c6b30080cf5000dd
:100b90000e00320020c6b30080cf500005003a009e
:100ba0000480fb0001002000020020000300200060
:100bb0000a00370040c7b30080cf50000300320066
:100bc0006640400080cf500006003a0004007800e4
:100bd000010020000200200003002000009cbe0055
:100be0000294be00081090000038a30014003200e8
:100bf0003800be002801be00e00f5000e08f580012
:100c0000e00f5900e08f59000d00320080c7b3009b
:100c100080cf54000300320080c5b30080cf540061
:100c200007003a007800900001c3b3000175780016
:100c30008000e80009f578000080e8007004980062
:100c4000780090000000450060049800894078001a
:100c50006d003700a8609000c0c4b30080cf500082
:100c600006003a009400780068805000000a78007e
:100c70005001be004000be0005003700940078001f
:100c800064805000000a78001000be0019080700b8
:100c9000009cbe000294be00380090000000e000fe
:100ca00003003d0078009000d1c2b3000a00370075
:100cb000081090000018a300030032007800900094
:100cc000b1c2b300040037000008a30005003200e1
:100cd0007800900001c2b300017578000000e800c0
:100ce00070049800780090000000450060049800af
:100cf000894078000800780033010700640037005d
:100d0000a8609000c0c6b30080cf5000250032001c
:100d10000a003c006440500080cf500028003200a0
:100d200000c0e80080cf500014003200684050003e
:100d300080cf500022003a000a00370040c7b300bd
:100d400080cf50001e0032006640400080cf50002f
:100d50001b0032006940500080cf500018003a005c
:100d6000060037001480e900000a780010007800bf
:100d7000485c900008487800450037001480e9007e
:100d8000000a78001002780068089000cf80de002a
:100d90000101780082017800009abe000292be0034
:100da0003b0037001480e900000a78001001780049
:100db00068089000cf80de000089be003400370054
:100dc0001480e900000a780010007800680c900098
:100dd000080878002e0037001180e90080087800ac
:100de00010007800cf80de000101780082017800d9
:100df000009cbe000294be007800900000004500f8
:100e00006004980081c7b30008007800170307004a
:100e10001f0037001480e900000a780010007800f5
:100e200060049800580990000200e00002003d00b4
:100e3000c6030700090037008000eb00ca03070063
:100e4000800078000000e00003003200680090009d
:100e5000008050000100370058089000100c9800e6
:100e60000b0037007800900002757800060037000c
:100e700078009000800045000904e00001003a007d
:100e800059c2b300894878000000e8007004980057
:100e90000000eb004f0578004f04be000000060084
:100ea0000400fa00889fbe008a9fbe008c1f780055
:100eb000000478000106780070089000f8009000a7
:100ec0000100500088089000010050009808900030
:100ed00001005000a808900001005000b8089000e0
:100ee00001005000c8089000810550000002220057
:100ef00090bf9f0000032300a0bf9f000810900038
:100f00000028a30018003a000b00e000160034008f
:100f10008b04780009057800e28f54000200360047
:100f20002a002000020037000900e0000b00340016
:100f300058009000c80190000a017800ee80570028
:100f400003000100500498000000e0009600320009
:100f50006808900000004500600c98008a845400e6
:100f60004240a900ebff3c00780190000200e00045
:100f70000b00340058009000c80190008c007800ed
:100f800003000100500498000000e00086003200d9
:100f900068089000f800900001004000600c980084
:100fa000880c90000900e000150034000905780065
:100fb000e28f5400020036002a00200002003700b1
:100fc0000900e0000b00340058009000c8019000b8
:100fd0000a017800ec8057000300010050049800db
:100fe0000000e0007000320068089000000045003a
:100ff000600c98008a8454004240a900ebff3c003a
:10100000180990000200e0000b003400e800900096
:1010100058009000c801900003000100500498009f
:101020000000e0006000320068089000980890001e
:1010300001004000600c9800a80c90000900e0003e
:101040001500340009057800e28f540002003600d4
:101050002a002000020037000900e0000b003400e5
:1010600058009000c80190000a017800ec805700f9
:1010700003000100500498000000e0004a00320024
:101080006808900000004500600c98008a845400b5
:101090004240a900ebff3c00380990000200e0004c
:1010a0000d003400e8009000180890008080400097
:1010b00058009000c80190000300010050049800ff
:1010c0000000e0003800320068089000b808900086
:1010d00001004000600c9800c80c90000900e0007e
:1010e0001500340009057800e28f54000200360034
:1010f0002a002000020037000900e0000b00340045
:1011000058009000c80190000a017800ec80570058
:1011100003000100500498000000e00022003200ab
:101120006808900000004500600c98008a84540014
:101130004240a900ebff3c00081090000028a300eb
:101140001b0032000b00e000190034008b04780013
:1011500009057800e28f5400020036002a002000c2
:10116000020037000900e0000b0034005800900036
:10117000c80190000a017800ee80570003000100ca
:10118000500498000000e00007003200680890005a
:1011900000004500600c98008a8454004240a90079
:1011a00003003400eaff37000080eb000100370045
:1011b0000000eb004f0678004f05be004f04be0054
:1011c0000080fa00000006008f04b000889fbe0077
:1011d0008a9fbe008c9fbe008e1f7800f0b79f00d4
:1011e00081f79f005001be004000be00f0979f00b5
:1011f000819f9f00929f9f00a39f9f0010c6b300f6
:101200000ff19700804f51001600320010c4b30058
:10121000804f510013003200ffb197005308900037
:101220000000e00003003d0060002000d0099800ad
:101230000c0037000000e0000a003a0070c6b3005e
:101240000ff29700804f52000300320070c4b300c9
:10125000804f520003003a0010002000ffb29700b8
:10126000d00a9800ffb09700c0fa2f000f0040008e
:10127000c702070080017800e20f500015003a0015
:1012800030002000ffb097009008980010c6b3000f
:101290000ff19700804f51000a0032006440400077
:1012a000804f5100070032000040e800804f51009d
:1012b00004003200219520000040e800804f5100da
:1012c00001003a0061952000ffb197006300900093
:1012d000160037000000e000180034003000200045
:1012e0007fb29700100a980010c6b3008ff29700e3
:1012f00080cf52000a0032006440400080cf52008c
:10130000070032000040e80080cf520004003200a5
:10131000a19520000040e80080cf520001003a0073
:10132000e19520007fb1970062009000315878006d
:101330003158780011487800c601370014c6b30050
:101340008ff2970084cf52000300320010c4b30024
:1013500080cf520013003a007fb0970060019000e8
:101360008200780000c3b30080587800ffb2970075
:10137000e102980080c7b3008ff2970084cf52003b
:101380000100320080c5b300804878000280e80088
:10139000ffb09700e0009800710090000080e80026
:1013a000f00098000300e00005003a00e3979f007a
:1013b00064fb2f000f01420003077800a0013700f3
:1013c00025962000e5b79f0010c6b3008ff0970068
:1013d00080cf50000500320010c4b30080cf500011
:1013e000a7003a0032972000e2b79f00ffb19700b4
:1013f000530890001e0220000000e00001003500ac
:101400000007e8000e02e800d4b79f006022b80091
:101410006033b8007f9097008f9897001f999700ce
:10142000af99970052060700ffb097003102be0047
:101430002103be000000e00004003d000400be00e7
:101440000601be0003f0a200020037000400be0047
:101450000601be00f0979f00819f9f00929f9f0012
:10146000a39f9f006f91970064015100e2979f0036
:10147000c3fa2f008f8141006a8041000048eb00d1
:101480006b824100c4b79f0031003700c2012000c9
:1014900003002000e5fa2f000f80420068020700d9
:1014a0007f9497008f9c97001f9d9700af9d97009a
:1014b0000800be000a01be00320607000006be009a
:1014c0005fb1970067015100d2b79f004240a90069
:1014d0000a003400570607000002be000203be00e7
:1014e0000800be000a01be0055060700f0979f00e5
:1014f000819f9f00929f9f00a39f9f00cfb1970065
:101500006780410071002000050037006f606600b1
:101510004c6add004466de000c067200c4eede009c
:10152000e00f5600e08f5e00050034008100e90006
:10153000e18f4000f5ff3a00010037000060eb004a
:101540008100e900fdff3b0067004000c0b79f003d
:10155000dfb297000500e000090034006022b80007
:101560006033b8007f9097008f9897001f9997007d
:10157000af999700340607000000e000c3ff3c006d
:1015800060fb2f008f0040004fb197000100510019
:101590000000e9008e0f500001003d0000077800b8
:1015a0000e00e00003003d0073fb2f000f8141009f
:1015b0002c003700800f570005003d000e804000d2
:1015c00010409000f3c0b300e74f500001003c0012
:1015d0008041eb00c4fa2f000f0242000e004200cf
:1015e0006a0040008e007800010037000000e9002a
:1015f0008100e90010417800834f5100fbff320069
:101600000107e800efcf510001003a000248e8006e
:101610000100e0000300350075fb2f000f81420040
:10162000060037000e07e8006f9097006400400046
:10163000e0979f0061fb2f000f8140008e0041006a
:101640008e017800030037001100fb006fb2970095
:10165000e44878008301e9008100e9000300e0002c
:10166000f9ff3d00ffb29700550890000000e00030
:10167000f3003d000e00e900d00a9800f0003700aa
:101680007f9497008f9c97001f9d9700af9d9700b8
:101690006022b8006033b8000800be000a01be0036
:1016a000b30507000000e00005003d000bf0a200bc
:1016b000f8979f00899f9f009a9f9f00ab9f9f0074
:1016c0006f909700725927000280b900026a2800c3
:1016d00013002000e1050700e4005000e1979f009f
:1016e00015003b00e3801000c0ff2f000084600065
:1016f0000800ea00e0979f007f9097008f9897007e
:101700001f999700af999700a99020000700370014
:101710000808a300030032003902be002903be00fe
:10172000dd0507000884d100e88444000800e000db
:10173000f7ff3c001b0037000100e0001d003400f3
:10174000c0ff2f0000806000e0979f000004780039
:101750006000b8000200200003ff2300a9902000d1
:10176000070037000808a300030032003902be005a
:101770002903be00c80507000884d100e88444009e
:101780000800e000f7ff3c000002be000203be00bc
:101790007f9097008f9897001f999700af999700b7
:1017a00032060700f0979f00819f9f00929f9f0045
:1017b000a39f9f00ffb097005109900060c6b3003f
:1017c0008ff1970080cf51000400320061002000ab
:1017d00060c4b30080cf510002003a006f929700be
:1017e000ea00420001074100f30f570001003400f6
:1017f0003e01200000c3b300e0779f0075fb2f007f
:101800008f824200b5b79f00330037000800be004a
:101810000a01be005b0507000006be00680757000e
:101820004240a9000e003400820507000002be00fd
:101830000203be000800be000a01be0080050700ca
:101840006022b80046782d00771924009205070021
:10185000f0979f00819f9f00929f9f00a39f9f00f2
:101860003fb0970068044000890020000d00370059
:10187000a4002000050020000c01be00e0fd2f00a8
:101880000f004000e70107007fa897008fb0970086
:101890001fb19700afb1970004c3b30004644100c7
:1018a0000006be00e00f5600e08f5e000600340028
:1018b0008904e900e18f4400edff3a00020037009f
:1018c00000c3b300006478008904e900fcff3b001a
:1018d00068044400b8b79f000e00e0000b0034001d
:1018e0007f9497008f9c97001f9d9700af9d970056
:1018f0006022b8006033b8000800be000a01be00d4
:10190000510507000000e000c0ff3c00c5fa2f00b1
:101910008f8242006a804200bfb097000080500072
:101920008001e9006f919700e70041006b81420060
:10193000010037000201e80000c3b300924f10001d
:10194000fcff320074fb2f000f004200808040003b
:10195000828050000080410002025000e1979f0009
:10196000ffb29700d509900060c6b3008ff29700d0
:1019700080cf52000300320060c4b30080cf520019
:1019800002003a008100e8000a00370050c6b300a8
:101990008ff0970080cf5000050032008000eb00f0
:1019a00050c4b3008ff2970080cf520001003a007c
:1019b00011002000018741008e0f520001003d0000
:1019c000040778000e00e0001d003500840f57006a
:1019d00005003d00e2407f0095c3b30040c3b30063
:1019e00080cf500001003c0005c3b3000e00410051
:1019f0008000e9008e017800010037008100e900d5
:101a00008301e90011427800854f5200fbff32004c
:101a10000307e80090c3b30080cf520001003a00f2
:101a20008448e8000300e00005003d000201e900f1
:101a30000e07e8006f9097000000e800e0979f0015
:101a40006f9297008e0178008ff097007fb097001b
:101a5000910107004f0778004f06be004f05be00fa
:101a60004f04be008f04b10000000600ef02b0007a
:101a7000889fbe008a9fbe008c9fbe008e1f78008c
:101a80000006780050992000c0b79f0080c5b300c1
:101a900080cf50000800320042982000c2b79f005b
:101aa0007740400080cf500003003a0083002000c0
:101ab000b3b79f000a00370080c7b30080cf500043
:101ac00005003200a4002000b4b79f0080c5b30019
:101ad00080cf500002003a0000012000b0b79f0004
:101ae0003c04be002c05be0040c6b30080cf5000b1
:101af000030032006540400080cf50000b003a00e8
:101b0000e00f5400e08f5c00e00f5d00e08f5d00af
:101b100006003d006000b8006011b80008045000e5
:101b2000898458000a0559008b855900e00f54003c
:101b3000e08f5c00e00f5d00e08f5d0004003a0084
:101b40005c0890008d0120000000e0000c003200d5
:101b5000bfb0970001027800cfa2de000503780035
:101b6000860378000800be000a01be001a060700be
:101b70004fb2970064407800d0df9f007d012000c5
:101b80003fb0970000027800cfa2de000503780086
:101b9000860378000800be000a01be0007060700a1
:101ba000009ebe000296be000d00e90061fc2f0001
:101bb0008f804000008740001e0037003fb1970033
:101bc00002047800cfc4de00090578008a05780099
:101bd0000802be000a03be007fa897008fb09700de
:101be0001fb19700afb19700ff050700d0b79f0066
:101bf000e1b79f00f2b79f0083bf9f008d06e90009
:101c00000802be000a03be007d0607007faa9700f7
:101c100000005200cfb09700615778005fb0970086
:101c2000efb097007fb197008fb99700009ebe007c
:101c30000296be003c00be002c01be00f0af9f002b
:101c400081b79f0092b79f00a3b79f00e00f50009d
:101c5000e08f5800e00f5900e08f59000200340077
:101c60000d00e000d5ff3c00bfb09700e88f5000aa
:101c700010003a000c1090000038a3000d00320054
:101c8000f78f560006003e0062fc2f000f01410056
:101c90008d00410000c3b300914f100005003200d9
:101ca0008d06e90000c3b30063fc2f008f81410063
:101cb00080f17e0078811600120e98006c00900072
:101cc00063fc2f008f8141008d80410029fa0700bd
:101cd0001c0990005c089000800f510006003d0038
:101ce00002005000000e98000c1090000040a1006f
:101cf000001698000f0037000000e0000d003d00c6
:101d00000c10900074006000f00f500009003a00c1
:101d10007c089000fc009000010050008c089000ae
:101d200001005000020050004240a90001003400b0
:101d3000000e98004f0778004f06be004f05be000a
:101d40004f04be00ef02b1000000060080007800e2
:101d5000010037000000e8001004e000fdff3a0039
:101d600001005000000006008001eb000400370075
:101d70008301e80090cf1000040032000000e8006a
:101d8000828f5100faff3a000000eb0000000600cd
:101d9000889fbe00800478006684400000ff270012
:101da000180060004401de00f07f2000800f510029
:101db0000e003a00800ceb00180478006f006400fd
:101dc0001c003a00210090000000e00019003a00d9
:101dd000110090000000e00016003a001000200002
:101de0001100e00014003200120037000200e00091
:101df00005003c0001007800db01070000017800cd
:101e00000000e00008003c00f0002800180060001e
:101e100001fe2300010c700020c02f00800c410047
:101e20000080eb0004003700800ceb000000eb00aa
:101e300001003700200020004f04be000000060013
:101e4000889fbe008a1f78008c9fbe000004780027
:101e50000206be00e6044000190178000200d0002e
:101e60004505de008a007800f07f2000800f5500d5
:101e70000c003a006f00610065003a0028009000f5
:101e80000000e00062003a00180090000000e0004e
:101e90005f003a00100020001800e0005d003200f2
:101ea0005b0037000a00e00007003a0008007800f5
:101eb000ad010700800078000000e000020034005f
:101ec0000a007800530037006108b9000c01400097
:101ed0008d814800e07f2000800f5100e08f590085
:101ee0000d0034001900e00004003d006000b8005f
:101ef0000200200003ff2f00030037006000b8003d
:101f00000200200003ff2700009cbe000294be00d8
:101f1000100020003f003700e00f5100e08f590013
:101f200005003400f000280019006000c410dd0036
:101f3000810c70003400370019007800010028007f
:101f4000010360006f0060000040a000800c78007a
:101f500061015100e0815900c0fc2f00f1ff2f000a
:101f6000800f5100818f59000d003d00860c7800d4
:101f70000000eb002004980010049800000c78008a
:101f8000240037008880e800110c780064004400c9
:101f90009008780019087800800ceb00700141006f
:101fa000f00f4100f7ff34008202ea001500320012
:101fb0008881e80070821200980078008508de00b1
:101fc000130078000400dd00008c70006401440000
:101fd000930078008508de00120078000400dd0020
:101fe00080897000920078008508de001900780072
:101ff0000400dd0000897000190078000500de0093
:10200000800c7800990c73000080eb000100370011
:10201000200020004f06be004f0578004f04be0090
:10202000000006000400fa00889fbe008a9fbe00e0
:102030008c1f78000006780092bf9f00a3bf9f000e
:102040000404be000401be001fb89700afb897009b
:10205000820307000005be000001be000800be00ac
:10206000950507001fb99700afb997000000510010
:102070008180590020069800310698000a8ebe0023
:102080000c0078004f0678004f05be004f04be00dc
:102090000080fa00000006000e00fa00889fbe00d3
:1020a0008a9fbe008c9fbe00000478000145780026
:1020b0000206780083047800840678000300e000bc
:1020c00002003c00190020002c9c200060c6b300d8
:1020d000804f55000e00320060c4b300804f5500a1
:1020e0000b00320070c6b300804f55000300320071
:1020f00070c4b300804f55009c003a00e48f460046
:102100008000350058089000808f56007d003d000b
:102110008d05e80060c6b300804f55001000320006
:1021200060c4b300804f55000d00320008109000cd
:102130000038a30004003a0058089000808f540033
:1021400001003d00590c9800580890000b00500009
:10215000500c980002003b000000eb00500c98006f
:102160000b00e00027003c00180990006800900078
:1021700001c3b300017079008201e800130c9800dc
:10218000580890000000e00003003c000810900098
:102190000038a3000500320068009000e1c2b300df
:1021a00001f079000280e800100c9800d808900037
:1021b0000b00ea00808f500001003d008105ea001d
:1021c0000b00ea00200c980001804500500c98009c
:1021d000890f500001003d0080047800390c980000
:1021e0006800900098089000010040000901780004
:1021f0008c007800dff807005808900009005000b4
:102200001a00370098089000680090008b8f5400e7
:1022100018003d0001004000090178008c007800a2
:10222000d4f807001808900000814400120c9800b0
:1022300009805500200c9800580890000000e0002c
:1022400003003c00081090000038a3000600320094
:10225000e8009000e0c2b300807079003808900078
:102260000000e800300c980058089000400c9800de
:10227000a6003700010040000b0178008c007800b8
:10228000bcf807001808900000814500120c980067
:102290008b845400580890000000e00003003c00cc
:1022a000081090000038a30005003200680090007c
:1022b000e1c2b300017079000200e800100c980040
:1022c00058089000890f500001003d0080047800fc
:1022d0006800900098089000010040008b004600c4
:1022e00009017800a3f80700180890000080440056
:1022f000100c98005808900009005000200c98001d
:102300008200370070c6b300804f550003003200d2
:1023100070c4b300804f550014003a005808900074
:10232000808f540004003d00081090000038a30086
:1023300001003a00590c9800580890000000e9008c
:10234000500c980002003b000000eb00500c98007d
:1023500070c6b300804f550002003a005ac6b30061
:102360000b0037005ac4b3000900370010c6b30091
:10237000804f550002003a000ac7b300040037003e
:1023800010c4b300804f550001003a000ac5b300e5
:1023900018099000680090003c7079008201e80004
:1023a000130c98000c027800580890000000e00020
:1023b00003003c00081090000038a3001700320012
:1023c000e8009000e0c2b30080f079008280e8006d
:1023d000110c9800580890000000e0000f00340035
:1023e0008904e900890f500001003d008004780055
:1023f00068009000008040000901780084007800a7
:102400005cf807001808900000804400100c980049
:102410005808900009005000200c980068009000b7
:1024200098089000010040000086e8000a587800f3
:10243000800078000d00e00004003500b0c2b30059
:10244000804878008c04780004003700d0c2b300c4
:10245000804878008c0478008d06ea008005eb0047
:102460000a003700a20020008d007800708057001d
:10247000890007000fb897009fb897007a81550030
:1024800001f17f008b05e800800678000d00e00078
:10249000f4ff3c00e18f550009003c0050c6b3003a
:1024a000804f55000300320050c4b300804f5500e8
:1024b00003003a0000c3b300005e78008c0478008b
:1024c0000b00e000040032000b00e900fa80570026
:1024d000008040000600370000c3b300805c780035
:1024e000050037008b05e90002c3b300a05c410082
:1024f0000b00e000fbff3c00680090009808900093
:102500000100400000805400300c9800081090003a
:1025100074006000f00f50000e003a007800900048
:102520009808900001004000a808900001004000b9
:10253000b808900001004000c808900081004000e9
:1025400078089000808f500002003d00010050008c
:10255000000c98004f06be004f05be004f04be00a1
:102560000080fa000000060000027800e602400049
:102570001500780001002800810360006f006000f2
:10258000800a780012003a00240090000000e00069
:102590000f003a00140090000000e0000c003a0028
:1025a000160020001400e000380032000800370058
:1025b000e4004200910a78000480e8009008780066
:1025c00014087800000aeb00700353000100370084
:1025d000160020001500e000f5ff32001300370060
:1025e0006401420080004000120078004f00de00cd
:1025f000808a70008481e800920078008180400029
:10260000130078004f00de0000897000930078000e
:1026100081804000140078004f00de008089700047
:1026200014007800000a40000603e9001500780055
:10263000ef0f5000eaff3600100037000481e80079
:102640009400d100120078004f00dd00008a700075
:10265000e40042009201d100110078004f00dd003b
:10266000008971001101d100150078004f00dd00d4
:1026700080087100950ad1000603e8001500780073
:10268000ff0f5000edff3e00ef0a6000958a7300d7
:10269000060078000000060002027800809fbe005d
:1026a000110009008200d800000178004f00be0030
:1026b00002a2b9008480500011009800020878003e
:1026c00000000600889fbe008a9fbe008c1f780015
:1026d0001a0107002101330003866c006450e100f9
:1026e000240032006420e100270032006150e10044
:1026f000220032006120e100210032008b8542007f
:10270000eb07b1000134b800003ab80008044200f9
:1027100089844a00013ab8000030b800888040003f
:1027200009014a0004003300000040008180480095
:10273000020149008b05e900c909dd008301700031
:102740000100320013002000c814de004814dd0030
:102750004709de001200b200c808de0008847000dd
:102760000e01070001f0a1000cf0a70001f0a0008d
:10277000030137006120e100050132000801be00bd
:102780000200be00f7ff37006150e100fcff3a0095
:10279000ff0037000001be00260107000470a700fb
:1027a00003f0a10003f8a30013003a006509b1008b
:1027b00010003200090035006928e10002003500f0
:1027c0000100280000000500000040008180480052
:1027d0008502e900fcff3a0000000600f88f420085
:1027e000050035008100d1000080d3008502e8009b
:1027f000fcff3a00000006008000eb00000005002e
:10280000889fbe008a9fbe00010578000100e0009d
:102810000400350008003c000000e0002000320009
:102820000500370060001000e080180002003b0047
:1028300001f02c001a0037000004be006011b8003f
:102840006b0920000982cf00020039000882cf0006
:102850000441b000694252000e00320008003b0003
:1028600082817100610164008904d1000884d30071
:102870008b05e8000442e800f9ff3a000500370044
:102880000804440089844c008b05e9000442e900f7
:10289000fbff3a00c10007000af0a70001f0a0000a
:1028a0004f05be004f04be000000060003f0a2006a
:1028b000889fbe008a9fbe008c1f78009f00070083
:1028c000a60033006450e1004f0032006420e100b4
:1028d0005200320003826c0007003b000905d00063
:1028e0000306d000820f54000c065d000200390080
:1028f00002003200890178000306780085825500c5
:1029000004003d000003fd008103fd008502ea0094
:102910008b854200840f720002003b0060001000b3
:10292000e08018006011b8000005eb007a28e10093
:102930000a00390006007800c75ddd00f707b20025
:10294000878075002d003700828171000a017800b0
:10295000610560008180d1000080d3008502e9001c
:10296000f9ff3b00060440008784480002003b005a
:1029700060041400e0841c000988a30007003200f2
:102980008a81710082817100610164008904d10033
:102990000884d3008b05e800170037000978a300ee
:1029a00013003a000b00e000130034008b05e9002f
:1029b0000804440089844c000a4474000978a30088
:1029c0000d003a000b00e000070034008b05e90021
:1029d0000804440089844c0001003a000b002000e8
:1029e0000978a300f7ff32000001eb000200370076
:1029f000828171000a017800680007000cf0a700ce
:102a000001f0a0005e0037006420e10002003a00ff
:102a1000838f6c005e0033000801be000200be0020
:102a200057003700f4ff2f009700370014002000f4
:102a300095003700889fbe008a9fbe008c1f7800db
:102a40003e0007004500330003866c006450e1003f
:102a50002e0032006420e100330032006150e100ba
:102a60002f0032006120e1003100320085855500e1
:102a7000eb07b00009002000080420000500370023
:102a80000804440089844c000a0031000603430016
:102a900087834b000001530081815b00f8ff330006
:102aa0000203be000800a0000804440089844c0012
:102ab000f6ff3900c639dd008301730001003200e2
:102ac000130020008904d1000884d3000998a300d2
:102ad000050032000800a7000300a0008904d1000f
:102ae0000884d3008b05e8008904d1000884d30052
:102af0000001eb000281d2002800070001f0a100d4
:102b00000cf0a70001f0a0001d0037006420e100d8
:102b10001f0032000801be000200be00f7ff3700b0
:102b20006120e1001a0032006000b800f3ff3700b6
:102b30000000200001f82700f0ff37000004be006d
:102b40003c0007000003be000405be000200be00fa
:102b500038000700844f7500000006000200be0028
:102b60006450e100050036006420e10002003600f8
:102b70000968a30001003a000800be000160a0003f
:102b80004f0678004f05be004f04be00000006004f
:102b9000f0ff2f00f1ff2700f9ff37008100200030
:102ba000618055000b003d000b00200061fe2f00ee
:102bb0000100e1001d0034008281710061016400a8
:102bc0008904d1000884d3000000e800faff3a002d
:102bd00071002000610064000300700002006000ca
:102be0000900320061044400e0844c000988a5001b
:102bf000050032008b05e8006808e10002003a0099
:102c00008904d1000884d300f20f20000258e100ab
:102c100005003d00c75ddd00f907b2008980750041
:102c200008007800000006000bf827008b007800f1
:102c300000000500c70ade00f107b200f50fb20080
:102c400008003200e1cf4200020032000170a00013
:102c500024000500810f7000010032000408050007
:102c600044000500810f700002003a0014000500c6
:102c70008502e9000000400081c04800fcff3b00e5
:102c80000170a00024000500889fbe008a9fbe003e
:102c9000841f7800a9ff07004f007800110033005f
:102ca000f0ff2f00838f6c0006003b0004056500d9
:102cb0000a00a7000800370009f0a6001000200055
:102cc00008003700820f5400838f5c000300390036
:102cd0001000200001003e000000200009f0a700c5
:102ce0000000ea004f05be004f04be000000e000f7
:102cf0000000060081037800ceff07000001be003f
:102d00006000b8000478a30013003a006220e100dc
:102d100015003e000d0039008301d1000281d3006f
:102d20008180d3008301d1000281d3008180d30050
:102d30008301d1000281d3008180d3000538b00027
:102d4000c42add00f300b2008381720007f0a700ff
:102d500003f0a00000000600f3ff2700f2ff2f00a1
:102d60006110b900fbff370003ff2700f7ff3700b2
:102d70008f1fd100560207008f87e9000000e00096
:102d8000000006001400fa00889fbe008a9fbe0063
:102d90008c9fbe000004be000205be006800470014
:102da0000a90be000890be00720207000070a700e3
:102db0000bf0a100304320009e0290008082520060
:102dc000b0fe2f000028e10011003d00b0fc2f00f4
:102dd0000028e100150034001e0990008e089000c4
:102de0007e0090000501b0000201d1008180d30077
:102df0000080d3008502e800fbff3a000b00e000f2
:102e000097023b0060001000e08018009402370039
:102e1000f0ff2f00f1ff27000b00e00090023b00c5
:102e200001002800000020008d0237006000b8007b
:102e30008b0237004f89de00820178008d02370057
:102e400007f0a200c2023700809feb0020020700bb
:102e50008f87e9000000e00000000600839f680003
:102e60000100e00002003d0060001000e08018005a
:102e70000300e00002003d0060011100e081190044
:102e8000300307004f00e00002003b00600010002c
:102e9000e0801800000006002800fa00889fbe00ad
:102ea0008a9fbe008c9fbe0003866b0058020700fd
:102eb0000028a30064003a000128a30067003a003c
:102ec0000008a30062003a000108a30065003a0070
:102ed0001e009000be08900081064000ed3fb1004a
:102ee000f4805700ee019000111ab8008e0990008e
:102ef000311bb8009e099000311cb800511db8006c
:102f0000f485570046000700fe0190003a000700d4
:102f10008b85e8003e0007008e0990004000070006
:102f2000ee019000340007008b85e80038000700b0
:102f30008e099000400007009e0990001b18b80001
:102f4000890440000a854800fe0190003400070013
:102f50008b85e80038000700ee0190003000070084
:102f60008e0990001b18b800890440000a854800ab
:102f70000a98a30008003a000402420085824a0031
:102f800006034b0087834b0008044c0089844c00e7
:102f90000a054d008d06e9008482720085027300e7
:102fa0004c3add008502720001003200150020005d
:102fb000443ade001400b2004538de00cb45dd00a7
:102fc0000b007000c540de00cb4ddd008b80700033
:102fd0004549de00cb55dd000b017100c551de0017
:102fe0000d037800e702070003f0a1000cf0a70032
:102ff00003f0a0001a0237001b18b8008502400039
:1030000006834800e0834b0060044c000700370053
:103010001b18b8000603400087834800faff3700fa
:103020001b18b8008703400008844800e0844c0067
:1030300060054d00000006001b18b80008044000a1
:1030400089844800faff37000108a30001023a0012
:103050005800be005801be00e3ff37000008a3007f
:10306000fc013a0009047800f9ff37002800fa0053
:10307000889fbe008a9fbe008c9fbe0003866b00a7
:10308000e30107006400e100440032006408e1004d
:103090004a0032006100e100460032006108e100b0
:1030a00049003200ec0647006000b8003d02be0057
:1030b0003d03be00f48657006011b8003d04be0019
:1030c0003d05be007d0320000b0037000000a0007e
:1030d0008d06e900130032000402420085824a0096
:1030e00006034b0087834b000000400081804800ae
:1030f00002014900838149000802520089825a0076
:103100000a035b008b835b00f0ff3b000802420078
:1031100089824a000a034b008b834b008d06e9002d
:10312000edff3a008482720086827200f707b200d7
:103130008782720001003200150020001e049000fa
:103140003e0b900006035400e63fb0000368a30066
:10315000070032000000a7000500a0008301d10095
:103160000281d3008180d3000080d3000603e800f1
:103170008301d1000281d3008180d3000080d3007d
:103180000002eb000482d2007e02070003f0a100df
:103190000cf0a70003f0a000b10137006402470063
:1031a0006408e100ab0132003400be003401be000f
:1031b000f6ff37006108e100a60132006011b80097
:1031c0006000b800f1ff370003ff27000200200075
:1031d000fbff3700881f7800000478005001be0014
:1031e0004000be0004004000858048000601490000
:1031f00087814900009cbe000294be000400e100eb
:103200000588e1000690e1000798e1000200310026
:10321000680044001008e8004f0478000000060031
:10322000f4874700889fbe008a9fbe008c9fbe0027
:103230008e1f78000205be000004be00d4b79f00b8
:10324000e5b79f00f6b79f0087bf9f000000eb0027
:10325000c0b79f00b0b79f00a0b79f0090b79f0076
:1032600080b79f000d042000bfb097004fb09700bb
:10327000000140000000e0000f003d004f08de00ac
:1032800000007100c0b79f009e00070001003d00d4
:1032900012002000a100070001003d0012002000e4
:1032a000a6000700b1000700b60007000f004000ad
:1032b000c8ff0700220037004f08de00000671003b
:1032c000ccb79f008f00070001003d0012002000d6
:1032d0009200070001003d00120020009700070047
:1032e000a20007000fb297009fb297002fb397007c
:1032f000bfb39700a90007000000520081805a0068
:1033000002015b0083815b0080b79f0091b79f0043
:10331000a2b79f00b3b79f000007eb009f00070014
:103320000020e10001a8e10002b0e10003b8e100e3
:10333000010031001e0020000e005600c0b79f00a3
:103340004fb297000400e000070035001000200095
:10335000010020006011b80008047000898470002a
:103360000a0571008b8571008d06e900beff3a00e9
:103370000400e00003003d00820007000f00400051
:1033800094ff07004fa897000000e00004003a00f7
:103390000fb497009fb497002fb59700bfb5970063
:1033a000940007004f0778004f06be004f05be008f
:1033b0004f04be004f01b10000000600881f7800d6
:1033c00018002000881f780095ff07008f87e9000c
:1033d0004f04780000000600801feb0090ff0700fc
:1033e0008f87e90000000600889fbe008a9fbe000c
:1033f0008c1f78006e00070007003d007300070077
:10340000e00f5b00e08f5b0007003d00320007002b
:103410000006eb00040037003400070002003d0006
:103420002a0007001c00200072000700e3ff0700cd
:103430000203be000002be000c00e00001003200ea
:10344000220007000400be000601be004f067800ff
:103450004f05be004f04be0000000600889fbe005e
:103460008a9fbe008c1f78005100070005003d00b8
:1034700056000700e00f5b00e08f5b0006003d0098
:10348000040037001900070003003d006000b80089
:103490006011b8001000070056000700ceff0700bb
:1034a0000203be000002be000c00e000010032007a
:1034b000060007000400be000601be004f067800ab
:1034c0004f05be004f04be00000006006000b800bb
:1034d0006011b800000037000402500085825800d7
:1034e0000603590087835900000006000006eb0020
:1034f000e00f5200e08f5a00e00f5b00e08f5b00ae
:10350000000006000180400090b79f000001eb0022
:103510008fb097000100e00000000600020070007c
:1035200090b79f000180400080b79f000001eb0032
:10353000ffa897000100e0000000060002007000f4
:1035400080b79f00018040006faa9700cf20de0067
:1035500001007000f0af9f00040242002500070048
:103560004f18de000002720000000600e4af9f006a
:103570000804440089844c000a054d008b854d00e9
:10358000000006003fb29700cfb297005fb39700ec
:10359000efb3970000fe2f00000006003fb0970039
:1035a000cfb097005fb19700efb197000000060021
:1035b0000205be000004be00e00f5000e08f58007e
:1035c000e00f5900e08f5900000006006000b800cd
:1035d0006011b80008045000898458000a05590099
:1035e0008b8559001c002000e00f5200e08f5a002c
:1035f000000006000800be000a01be000000060030
:10360000889fbe008a9fbe008c1f78000205be0006
:103610000004be000006eb00e00f5000e08f5800f1
:10362000e00f5900e08f590007003d006000b8002e
:103630006011b80008045000898458000a05590038
:103640008b8559001c002000e00f5200e08f5a00cb
:10365000e00f5b00e08f5b0002003d000f00070001
:103660000c00a2000800be000a01be0071010700a4
:103670000203be000002be000c00e00001003200a8
:10368000060007000400be000601be004f067800d9
:103690004f05be004f04be00000006006000b800e9
:1036a0006011b800040250008582580006035900da
:1036b0008783590000000600020ab900001bb90008
:1036c0000200b800810042008100430000000600b3
:1036d000889fbe008a9fbe008c9fbe000404be006f
:1036e0000605be00809fbe00829fbe0073010700da
:1036f000040678000800be000a01be006f01070042
:10370000840678004f03be004f02be008d4f760046
:103710007fb0970013003300f0ff2f008b8f6b00fa
:1037200006003b000d0666000c00a7000a003700eb
:1037300007f0a600100020000a003700880f520092
:10374000898f5a008a0f5b008b8f5b000300390062
:103750001000200001003e000000200007f0a7003c
:103760000000ea004f06be004f05be004f04be0039
:1037700000000600800078005002be005003be002a
:103780004439de00f700b200f37f2000030161003e
:10379000090032000218e10016003a0085017200ab
:1037a00083017300838173000008200015003a0034
:1037b0004000200013003700850172008301730070
:1037c0008381730005003a0004a8be0006a8be006d
:1037d000100020000b0037000201e9000402420043
:1037e00085824a0006034b0087834b000748a300ed
:1037f000f9ff32000740a00004a8be0006a8be00e2
:103800002000200080009800920098000000060030
:10381000680447000294be000094be00fc04470008
:103820008694be008494be0009007800d1ff070092
:1038300008007800cfff070099007800814f7000e2
:103840000b003b000800be002e0107004f00b10036
:1038500003003700f3ff2700f2ff2f006110b900cb
:103860004f06be004f05be004f04be000080fa00a8
:1038700000000600889fbe00830478000300e0007b
:103880002c00350003003c0000827000040271002f
:103890002600320036432000c50020008383cf007d
:1038a0000a0039000541b1008283cf0007003900ca
:1038b0000541b1008183cf00040039000541b1000a
:1038c0008083cf00010039000541b10085c353005a
:1038d0006022b800120032000a003b0084827200ad
:1038e000610260008301d1000281d3008180d30096
:1038f0000080d3000603e8008743e800f7ff3a00a2
:1039000007003700000040008180480002014900a4
:10391000838149000603e9008743e900f9ff3a0083
:103920009800070009f0a70003f0a0004f04be00b4
:103930000000060060001000e0801800600119001f
:10394000e0811900d3ff3b00033e2c00f7ff370056
:103950002800fa00889fbe008a9fbe008c9fbe0090
:1039600007067800878669000c003b000304780096
:103970008704780008f0a10009f0a100840f50002e
:10398000858f5800860f5900890f5c0003003300b3
:103990000cf0a20001003a000cf0a1009cff07000f
:1039a0006400e1005f003200780147006408e10034
:1039b000610032006c014700748557003200be0080
:1039c0001201be003a04be001a05be001e0390009c
:1039d000be0a90008503530006003d000004fd0070
:1039e0008104fd000205fd008305fd008703ea0058
:1039f000050378000df8a3000400320060041400f1
:103a0000e0841c0060051d00e0851d006022b800f8
:103a10007d0320000d38e1008006eb000b0039002b
:103a20004433dd00f300b200830173003900370036
:103a3000848272000d027800e10664008b85d1005b
:103a40000a85d3008984d3000884d3008703e90062
:103a5000f7ff3b0008004000898048000a01490048
:103a60008b81490004003b0060001000e0801800da
:103a700060011900e08119000358a3000900320019
:103a80008d82720084827200610260008301d10025
:103a90000281d3008180d3000080d3000603e800b8
:103aa0001b0037000348a30017003a000600e0009f
:103ab000170034000603e9000d00a30000004800d1
:103ac0008180480002014900838149000348a30026
:103ad0000f003a000600e000090034000603e90088
:103ae00000004000818048000201490083814900b4
:103af00001003a000003eb000348a300f5ff320089
:103b00006022b80002003700848272006182660081
:103b10001c00070003f0a1000cf0a70003f0a000b8
:103b20004fff3700640147006408e10002003a00db
:103b30000df8a30047ff3a003200be001201be009c
:103b400047ff37006022b800060220000000d000c6
:103b50008180d2000482d2008582d2000000a000c1
:103b60000202520083825a00030031000202420026
:103b700083824a000000a1000603e900f3ff3a0037
:103b80000000060018002000570020000804530021
:103b90000d003d000600200097fc2f000740e100cb
:103ba0001e00340084827200610260008301d10033
:103bb0000281d3008180d3000080d3000804e80094
:103bc000f8ff3a004700200061046000050474001b
:103bd000040464000d00320061004000e0804800f1
:103be00060014900e081490003b8a50007003200e8
:103bf0000603e8006538e10004003a008301d100c3
:103c00000281d3008180d3000080d300f87f2000a0
:103c10000830e10003003500080378006000b800b8
:103c20006011b8004433dd00f300b200830173007b
:103c300000000600889fbe008a9fbe008c9fbe00c9
:103c40000404b8000506b8008904460060854e00eb
:103c50000606b8000a054600e0854e000706b800d3
:103c60008b054600040eb800890446000a854e0004
:103c7000e0854d00050eb8000a0546008b854e0014
:103c8000060eb8008b0546000416b8000a0546006b
:103c90008b854e000516b8008b054600041eb80043
:103ca0008b0546000800be000a01be004f06be009c
:103cb0004f05be004f04be000000060005ff2700b0
:103cc00005826100070032000428e1000100320093
:103cd000240005000600070001003a00440005002a
:103ce0000408050002000700f9ff3a00140005006f
:103cf0006f8261008102700085027100850272008e
:103d000000000600e48240001078a30007003200a3
:103d1000640240001178a3003400be001401be000c
:103d2000040032000330a700000006003500be008a
:103d30001501be000330a000000006000000fa00dc
:103d400023c2bf000004a2000000fb00610060006d
:103d50000080fa00000006000000fa0033c2bf0035
:103d60000004a2000000fb00610060000080fa0077
:103d7000000006000000fa0021e2a9009560a900f9
:103d80009580a9008560a9008580a9000080fa00bf
:103d9000000006000000fa0031e2a90097c0a90067
:103da00097e0a90087c0a90087e0a9000080fa0079
:103db000000006000200fa00000f78008560a900ec
:103dc0008580a9001e0078006740600067406000a1
:103dd00067406000674060004401dd00910a2000f8
:103de00091407800f0c8b30000c06000024070004d
:103df000a9e0b700000720001e0060004400de00bc
:103e00006740600067416000a10a2000914078008f
:103e100080cfb30000c0600002407000aae0b7008d
:103e20009e007800688060004300de006140600012
:103e3000614060004301dd0051092000914078009d
:103e400070cfb30000c060000240700095e0b70082
:103e5000000820001e0060004700de006140600096
:103e6000614060004401dd0051092000914078006c
:103e7000f0ceb30000c060000240700095e0b700d3
:103e80000080fa00000006000200fa00000f78002f
:103e900087c0a90087e0a9001e0078006740600085
:103ea000674060006740600067416000310b2000a0
:103eb0009140780080cfb30000c0600002407000e5
:103ec000b3e0b700000720001e0060004400de00e1
:103ed00067406000674060004401dd00310b200056
:103ee00091407800f0c8b30000c06000024070004c
:103ef000b3e0b7009e007800688060004300de00f9
:103f000061406000614060004601dd0071092000f1
:103f100091407800f0cbb30000c060000240700018
:103f200097e0b700000820001e0060004700de0098
:103f300061406000c700dd0097c0bf000074a100b1
:103f40000140700097e0b7000080fa000000060012
:103f50000000fa0022c2bf00614060000080fb0048
:103f60000080fa00000006000000fa0032c2bf0024
:103f7000614060000080fb000080fa000000060045
:103f80000c00fa00200798003107980042079800bb
:103f90000000eb00100798003e009000000f780032
:103fa000230037009e0090004e009000808f50004c
:103fb000040031001e0090000000e8001007980087
:103fc000030037002e009000500798001d003700b6
:103fd000dfff07000004e000f2ff32000000eb000a
:103fe0001007980020c2bf0066406000e64f5000f6
:103ff00007003a00311180003e009000010878006f
:104000003e0090000080e80030079800050037006f
:1040100030118000804078001e0078000148780050
:104020001e0fe8002e0090000000e9002007980015
:104030002e0090000000e000e5ff3a002e00900006
:10404000500798005e0090000080fa000000060013
:104050000c00fa00200798003107980042079800ea
:104060000000eb00100798003e009000000f780061
:10407000230037009e0090004e009000808f50007b
:10408000040031001e0090000000e80010079800b6
:10409000030037002e009000500798001d003700e5
:1040a000b1ff07000004e000f2ff32000000eb0067
:1040b0001007980030c2bf0066406000e64f500015
:1040c00007003a00b11180003e009000010878001e
:1040d0003e0090000080e80030079800050037009f
:1040e000b0118000804078001e0078000148780000
:1040f0001e0fe8002e0090000000e9002007980045
:104100002e0090000000e000e5ff3a002e00900035
:10411000500798005e0090000080fa000000060042
:104120000600fa00000f7800110798002207980097
:104130002e009000401188001e00780000118800b9
:104140001e009000101188000080fa000000060098
:104150000600fa00000f7800110798002207980067
:104160002e009000c01188001e0078008011880089
:104170001e009000901188000080fa0000000600e8
:104180000400fa00100798001e009000000f78004d
:1041900023c2bf00624060000004e000fcff3a0060
:1041a00020c2bf0066406000e64f500019003a0090
:1041b0000a0037001e0090001000780020118800cf
:1041c0001e0090000080e8001007980023c2bf0086
:1041d000624060000004e000fcff3a001e00900016
:1041e000100078000000e000f2ff3a000d003700f8
:1041f0001e007800104078000000fb0020118800ad
:104200001e0fe80023c2bf00624060000004e0000f
:10421000fcff3a001e007800104078000004e00027
:10422000f3ff3a000080fa00000006000400fa00e4
:10423000100798001e009000000f780033c2bf00e6
:10424000624060000004e000fcff3a0030c2bf00a2
:1042500066406000e64f500019003a000a0037003f
:104260001e00900010007800a01188001e00900031
:104270000080e8001007980033c2bf006240600071
:104280000004e000fcff3a001e00900010007800df
:104290000000e000f2ff3a000d0037001e00780039
:1042a000104078000000fb00a01188001e0fe800fd
:1042b00033c2bf00624060000004e000fcff3a002f
:1042c0001e007800104078000004e000f3ff3a0080
:1042d0000080fa00000006000200fa0020c2bf00c1
:1042e00066406000e64f500003003a003011800045
:1042f000000f78000400370031118000f00f20001b
:1043000080806000010f78001e0078000080fa00b5
:10431000000006000200fa0030c2bf0066406000e4
:10432000e64f500003003a00b0118000000f780003
:1043300004003700b1118000f00f20008080600081
:10434000010f78001e0078000080fa0000000600cf
:104350000200fa00000f780023c2bf006240600034
:104360000004e000fcff3a0020c2bf00664060008d
:10437000e64f500003003a001e007800201188002c
:1043800003003700f00f20001e006000201188009d
:104390000080fa00000006000200fa00000f78001a
:1043a00033c2bf00624060000004e000fcff3a003e
:1043b00030c2bf0066406000e64f500003003a0084
:1043c0001e007800a011880003003700f00f2000c5
:1043d0001e006000a01188000080fa0000000600a6
:020000040000fa
:0200000401f009
:04000000ffff0000fe
:020000040000fa
:0200000401f009
:04000400ffff0000fa
:020000040000fa
:0200000401f009
:04000c00faff0000f7
:020000040000fa
:0200000401f009
:040010007eff00006f
:020000040000fa
:0200000401f009
:040014007fff00006a
:020000040000fa
:0200000401f009
:04001800ffff0000e6
:020000040000fa
:10000800a4420000583a00006e3a0000843a00000a
:100018009a3a0000a4420000a4420000a442000052
:10002800a4420000a4420000a4420000a442000030
:10003800a4420000a4420000a4420000a442000020
:10004800a4420000a4420000a4420000c0410000f5
:100058005e410000a4420000a4420000a442000047
:10006800a442000002380000a4420000a44200009c
:10007800a4420000a4420000a4420000a4420000e0
:10008800a4420000a4420000a4420000a4420000d0
:10009800a4420000a4420000fe410000fc40000011
:1000a800a4420000a4420000a4420000a4420000b0
:1000b800a4420000a4420000a4420000a4420000a0
:1000c800a4420000a4420000a4420000a442000090
:1000d800a4420000a4420000a4420000a442000080
:1000e800a4420000a4420000a4420000a442000070
:1000f800a4420000a4420000a4420000a442000060
:10010800a4420000a4420000a4420000a44200004f
:10011800a4420000a4420000a4420000a44200003f
:10012800a4420000a4420000a4420000a44200002f
:10013800a4420000a4420000a4420000a44200001f
:10014800a4420000a4420000a4420000a44200000f
:10015800a4420000a4420000a4420000a4420000ff
:10016800a4420000a4420000a4420000a4420000ef
:10017800a4420000a4420000a4420000a4420000df
:10018800a4420000a4420000a4420000a4420000cf
:10019800a4420000a4420000a4420000a4420000bf
:1001a800a4420000a4420000a4420000a4420000af
:1001b800a4420000a4420000a4420000a44200009f
:1001c800a4420000a4420000a4420000a44200008f
:1001d800a4420000a4420000a4420000a44200007f
:1001e800a4420000a4420000a4420000a44200006f
:0801f800a4420000a442000033
:020000040000fa
:10020800a4420000583a00006e3a0000843a000008
:100218009a3a0000a4420000a4420000a442000050
:10022800a4420000a4420000a4420000a44200002e
:10023800a4420000a4420000a4420000a44200001e
:10024800a4420000a4420000a4420000c0410000f3
:100258005e410000a4420000a4420000a442000045
:10026800a442000002380000a4420000a44200009a
:10027800a4420000a4420000a4420000a4420000de
:10028800a4420000a4420000a4420000a4420000ce
:10029800a4420000a4420000fe410000fc4000000f
:1002a800a4420000a4420000a4420000a4420000ae
:1002b800a4420000a4420000a4420000a44200009e
:1002c800a4420000a4420000a4420000a44200008e
:1002d800a4420000a4420000a4420000a44200007e
:1002e800a4420000a4420000a4420000a44200006e
:1002f800a4420000a4420000a4420000a44200005e
:10030800a4420000a4420000a4420000a44200004d
:10031800a4420000a4420000a4420000a44200003d
:10032800a4420000a4420000a4420000a44200002d
:10033800a4420000a4420000a4420000a44200001d
:10034800a4420000a4420000a4420000a44200000d
:10035800a4420000a4420000a4420000a4420000fd
:10036800a4420000a4420000a4420000a4420000ed
:10037800a4420000a4420000a4420000a4420000dd
:10038800a4420000a4420000a4420000a4420000cd
:10039800a4420000a4420000a4420000a4420000bd
:1003a800a4420000a4420000a4420000a4420000ad
:1003b800a4420000a4420000a4420000a44200009d
:1003c800a4420000a4420000a4420000a44200008d
:1003d800a4420000a4420000a4420000a44200007d
:1003e800a4420000a4420000a4420000a44200006d
:0803f800a4420000a442000031
:020000040000fa
:1043e00000000000000000000000000000000000cd
:1043f000004900006e69000074690000616c0000f3
:1044000069730000696e000067200000414e0000e3
:10441000414c00004f4700000a0d00000049000019
:104420006e69000074690000616c0000697300002f
:10443000696e00006720000053500000490a000028
:104440000d000000496e0000697400006961000001
:104450006c690000736900006e670000204900006d
:10446000324300000a0d000000570000616900009f
:10447000746900006e670000206600006f72000023
:10448000204900004d5500000a0d000000490000c1
:104490004d550000204900007320000052650000c7
:1044a00061640000793a000020250000730a0000d2
:1044b0000d250000635b0000324a0000002500006b
:1044c000635b0000324a0000256300005b3b000094
:1044d000484200006f610000726400002025000067
:1044e000730a000045520000202500002b2e00001a
:1044f00032660000202500002b2e000032660000ee
:10450000202500002b2e0000326600000a45000026
:1045100046200000252b00002e32000066200000ff
:10452000252b00002e32000066200000252b000005
:104530002e320000660a00004143000020250000e2
:104540002b2e000032660000202500002b2e0000dc
:1045500032660000202500002b2e0000326600008d
:104560000a47000052200000252b00002e320000d8
:1045700066200000252b00002e320000662000007f
:10458000252b00002e320000660a00004d47000077
:10459000202500002b2e00003266000020250000a0
:1045a0002b2e000032660000202500002b2e00007c
:1045b000326600000a41000054200000252b000054
:1045c0002e32000066200000252b00002e32000055
:1045d000660a0000434c0000202500002b2e00003e
:1045e00032660000202500002b2e000032660000fd
:1045f000202500002b2e0000326600000a0000007b
:020000040000fa
:104600000400fa00204798000040eb00004f7800bb
:10461000ae40900000c1b300d10b0700004f7800fe
:104620001e00fb000080fa00000006000400fa00f3
:1046300020479800314798000040eb00004f780079
:104640003e419000ae40900000c1b3001c0c07003a
:10465000004f78001e00fb000080fa0000000600fa
:104660000c00fa0010079800210798000000eb00ea
:10467000000f78002e0090000000e00003003a00d8
:10468000e0ff2f00500798001c00370010002000aa
:10469000300798000a0037003e0090008000780044
:1046a0001e00900000804000104078000080fb0059
:1046b0001e0f40003e0090000000e8003007980008
:1046c000be0090002e009000808f5000f2ff390055
:1046d000f00f20001e0f60001e00e00003003200fb
:1046e0000080eb0040079800020037000000eb005c
:1046f000400798004e009000500798005e00900020
:104700000080fa00000006001800fa00200f980050
:10471000e3004700a3c0b30042c7b30000c1b30029
:10472000b30b0700204798002e4090000004e000e3
:10473000040032002e4090000000fb00300f980073
:104740001d00370063004700a1002000c4ff0700e0
:10475000204798002e4090000004e0000400320042
:104760002e4090000000fb00300f98001200370030
:104770000000eb00000f7800090037001e007800f1
:10478000800078002e089000008140009e00e80024
:104790006300470061407800004978001e0fe80080
:1047a000700020009e0f1000f4ff34002e40900097
:1047b0000000fb00300f98003e0890000080fa00d7
:1047c000000006000600fa00100798000040eb0009
:1047d000004f7800e3c0b300e2c0b3009e00900039
:1047e00000c1b300820b0700004f78001e04e000f8
:1047f000030032001e00fb00200798000b0037006a
:104800001e009000e100200095ff0700004f780097
:104810001e04e000030032001e00fb002007980089
:10482000020037000000eb00200798002e009000e7
:104830000080fa00000006000600fa001007980049
:104840000040eb00004f7800e3c0b3000041eb00f4
:104850009e00900000c1b300650b0700004f780078
:104860001e04e000030032001e00fb002007980039
:104870000b0037001e009000e100200078ff0700c9
:10488000004f78001e04e000030032001e00fb0011
:1048900020079800020037000000eb002007980076
:1048a0002e0090000080fa00000006000600fa00ca
:1048b000100798000040eb00004f7800e3c0b30001
:1048c000c2c1b3009e00900000c1b300480b0700b6
:1048d000004f78001e04e000050032009e40780082
:1048e0006ac050000000fb00200798000d00370050
:1048f0001e009000e100200059ff0700004f7800e3
:104900001e04e00005003200e0ccb3001e40400071
:104910000000fb0020079800020037000000eb00b9
:10492000200798002e0090000080fa00000006008a
:104930000600fa00100798000040eb00004f7800d6
:10494000e3c0b300a2c2b3009e00900000c1b30058
:10495000270b0700004f78001e04e0000300320020
:104960001e00fb00200798000b0037001e0090007f
:10497000e10020003aff0700004f78001e04e0002d
:10498000030032001e00fb002007980002003700e1
:104990000000eb00200798002e0090000080fa0035
:1049a000000006000600fa00100798000040eb0027
:1049b000004f7800e3c0b30082c3b3009e009000b4
:1049c00000c1b3000a0b0700004f78001e04e0008e
:1049d000030032001e00fb00200798000b00370088
:1049e0001e009000e10020001dff0700004f78002e
:1049f0001e04e000030032001e00fb0020079800a8
:104a0000020037000000eb00200798002e00900005
:104a10000080fa00000006000600fa001007980067
:104a20000040eb00004f780063c0b30062c4b300e5
:104a30009e00900000c1b300ed0a0700004f78000f
:104a40001e04e000030032001e00fb002007980057
:104a50000b0037001e0090006100200000ff0700df
:104a6000004f78001e04e000030032001e00fb002f
:104a700020079800020037000000eb002007980094
:104a80002e0090000080fa00000006000600fa00e8
:104a9000100798000040eb00004f780063c0b3009f
:104aa000c2c4b3009e00900000c1b300d00a07004a
:104ab000004f78001e04e000030032001e00fb00df
:104ac000200798000b0037001e00900061002000b6
:104ad000e3fe0700004f78001e04e00003003200f0
:104ae0001e00fb0020079800020037000000eb00ca
:104af000200798002e0090000080fa0000000600b9
:104b00000600fa00100798000040eb00004f780004
:104b100043c1b30002c6b3009e00900000c1b300c1
:104b2000b30a0700004f78001e04e00005003200c1
:104b30009e4078006ac050000000fb0020079800eb
:104b40000d0037001e00900041012000c4fe070048
:104b5000004f78001e04e00005003200e0ccb300f6
:104b60001e4040000000fb002007980002003700b4
:104b70000000eb00200798002e0090000080fa0053
:104b8000000006000600fa00100798000040eb0045
:104b9000004f7800e3c0b30022c5b3009e00900030
:104ba00000c1b300920a0700004f78001e04e00025
:104bb000030032001e00fb00200798000b003700a6
:104bc0001e009000e1002000a5fe0700004f7800c5
:104bd0001e04e000030032001e00fb0020079800c6
:104be000020037000000eb00200798002e00900024
:104bf0000080fa00000006000600fa001007980086
:104c00000040eb00004f780023c1b30062c6b30040
:104c10009e00900000c1b300750a0700004f7800a5
:104c20001e04e000030032001e00fb002007980075
:104c30000b0037001e0090002101200088fe0700b5
:104c4000004f78001e04e000030032001e00fb004d
:104c500020079800020037000000eb0020079800b2
:104c60002e0090000080fa00000006000200fa000a
:104c7000000f7800e0c0b30061fe070080407800bc
:104c80001e007800014878001e0fe800f0c0b30055
:104c90005bfe0700804078001e0078000148780025
:104ca0001e0fe80000c1b30055fe070080407800e9
:104cb0001e007800014878001e0fe80010c1b30004
:104cc0004ffe0700804078001e0078000148780001
:104cd0001e0fe80020c1b30049fe070080407800a5
:104ce0001e007800014878001e0fe80030c1b300b4
:104cf00043fe0700804078001e00780001487800dd
:104d00001e0fe80040c1b3003dfe07008040780060
:104d10001e007800014878001e0fe80050c1b30063
:104d200037fe0700804078001e00780001487800b8
:104d30001e0fe80060c1b30031fe0700804078001c
:104d40001e007800014878001e0fe80070c1b30013
:104d50002bfe0700804078001e0078000148780094
:104d60001e0fe80080c1b30025fe070080407800d8
:104d70001e007800014878001e0fe80090c1b300c3
:104d80001ffe0700804078001e0078000148780070
:104d90001e0fe800a0c1b30019fe07008040780094
:104da0001e007800014878001e0fe800b0c1b30073
:104db00013fe0700804078001e007800014878004c
:104dc0000080fa0000000600cc00fa0050a798000e
:104dd0000000eb00000f78005ea090006100600012
:104de0000004e0002b0032000e80e80075fe070092
:104df0000000fb001e0f70000e80e80010419000c4
:104e00000e80e800204290000e80e800b040900044
:104e10000e80e80040409000824178000441780014
:104e20005002070000408800114088000e80e80012
:104e3000504190000e80e800604290000e80e80033
:104e4000f04090000e80e800004890008241780019
:104e50000441780043020700204088003140880068
:104e60000e80e800104990000e80e800204a900073
:104e70000e80e800b04890000e80e80040489000a6
:104e800082417800044178003602070040408800e3
:104e9000514088005ea090004800de006100600084
:104ea0000004e0002b0032000e80e80062fe0700e4
:104eb0000000fb001e0f70000e80e8001041900003
:104ec0000e80e800204290000e80e800b040900084
:104ed0000e80e80040409000824178000441780054
:104ee0002002070060408800714088000e80e800c2
:104ef000504190000e80e800604290000e80e80073
:104f0000f04090000e80e800004890008241780058
:104f10000441780013020700804088009140880017
:104f20000e80e800104990000e80e800204a9000b2
:104f30000e80e800b04890000e80e80040489000e5
:104f4000824178000441780006020700a0408800f2
:104f5000b14088005ea090000000d10061006000b8
:104f60000004e0002b0032000e80e8004ffe070036
:104f70000000fb001e0f70000e80e8001041900042
:104f80000e80e800204290000e80e800b0409000c3
:104f90000e80e80040409000824178000441780093
:104fa000f0010700c0408800d14088000e80e80072
:104fb000504190000e80e800604290000e80e800b2
:104fc000f04090000e80e800004890008241780098
:104fd00004417800e3010700e0408800f1408800c8
:104fe0000e80e800104990000e80e800204a9000f2
:104ff0000e80e800b04890000e80e8004048900025
:105000008241780004417800d60107000041880001
:10501000114188005ea090004200de006100600047
:105020000004e0002b0032000e80e80040fe070084
:105030000000fb001e0f70000e80e8001041900081
:105040000e80e800204290000e80e800b040900002
:105050000e80e800404090008241780004417800d2
:10506000c001070060418800714188000e80e8009f
:10507000504190000e80e800604290000e80e800f1
:10508000f04090000e80e8000048900082417800d7
:1050900004417800b30107008041880091418800f5
:1050a0000e80e800104990000e80e800204a900031
:1050b0000e80e800b04890000e80e8004048900064
:1050c0008241780004417800a6010700a0418800d1
:1050d000b14188005ea090004300de0061006000e6
:1050e0000004e0002b0032000e80e800a5fe07005f
:1050f0000000fb001e0f70000e80e80010419000c1
:105100000e80e800204290000e80e800b040900041
:105110000e80e80040409000824178000441780011
:105120009001070040418800514188000e80e8004e
:10513000504190000e80e800604290000e80e80030
:10514000f04090000e80e800004890008241780016
:105150000441780083010700a0418800b141880024
:105160000e80e800104990000e80e800204a900070
:105170000e80e800b04890000e80e80040489000a3
:10518000824178000441780076010700a040880041
:10519000b14088005ea090004400de006100600025
:1051a0000004e0002b0032000e80e800fdfd070047
:1051b0000000fb001e0f70000e80e8001041900000
:1051c0000e80e800204290000e80e800b040900081
:1051d0000e80e80040409000824178000441780051
:1051e0006001070020428800314288000e80e800fc
:1051f000504190000e80e800604290000e80e80070
:10520000f04090000e80e800004890008241780055
:105210000441780053010700404288005142880051
:105220000e80e800104990000e80e800204a9000af
:105230000e80e800b04890000e80e80040489000e2
:1052400082417800044178004601070060428800ee
:10525000714288005ea090004500de0061006000a1
:105260000004e000110032000e80e80007fe070095
:105270000000fb001e0f70000e80e800104190003f
:105280000e80e800204290000e80e800b0409000c0
:105290000e80e80040409000824178000441780090
:1052a0003001070040418800514188005ea0900015
:1052b0004600de00610060000004e00011003200e2
:1052c0000e80e800d4fd07000000fb001e0f7000f8
:1052d0000e80e800104190000e80e800204290000f
:1052e0000e80e800b04090000e80e8004040900042
:1052f00082417800044178001a010700804288004a
:10530000914288005ea090004700de0061006000ce
:105310000004e000380032000e80e80036fe07008e
:105320000000fb001e0f70000e80e800104190008e
:105330000e80e800204290000e80e800b04090000f
:105340000e80e800404090008241780004417800df
:1053500004010700a0428800b14288000e80e800e6
:10536000504190000e80e800604290000e80e800fe
:10537000f04090000e80e8000048900082417800e4
:1053800004417800f7000700c0428800d14288003d
:105390000e80e800104990000e80e800204a90003e
:1053a0000e80e800b04890000e80e8004048900071
:1053b0008241780004417800ea000700e04288005a
:1053c000f14288000e80e800504990000e80e8000d
:1053d000604a90000e80e800f04890000e80e800df
:1053e000005090008241780004417800dd00070001
:1053f00000438800114388001e0078000080fa00f6
:10540000000006000e00fa004007980051079800bf
:105410004e0090000000e800300798000000eb000c
:10542000100798004e0090005efd07000000fb0092
:10543000000f78001e00e0000400320080f32f000f
:105440001e004000600798002d0037004e009000bd
:1054500010407800e14f500003003e000000eb00d8
:1054600060079800260037004e009000104078003a
:105470000080fb000080e9000080d1001007980048
:105480000000eb0020079800170037003e00900056
:10549000104078008081fb003e0090000000e80092
:1054a000300798003e009000104078000081fb001b
:1054b0003e0090000000e800300798002e009000a9
:1054c00000004000800078005e0090008080400076
:1054d0004810dd0003007000800878002e00900066
:1054e0000000e80020079800ae0090001e00900029
:1054f000808f5000e5ff39001e0090006007980083
:105500006e0090000080fa00000006000600fa001d
:10551000404798004e409000004f78001a00370036
:10552000803e20001007980010003700cbc2bf005b
:10553000624060000004e00005003a00cb22a800b1
:1055400000f4210001002000f10b070004003700e7
:10555000cb22a90000f4210001002000ec0b070081
:105560001e0090000000e900100798001e00900047
:105570000000e000edff3a0000902000d103200081
:10558000e30b07001e4fe9001e04e000e4ff3a00b1
:105590000080fa00000006000400fa0000d4200099
:1055a00031002000008fbe0011003700cbc2bf00c9
:1055b000624060000004e00005003a00cb22a80031
:1055c00000f4210001002000d10b07000400370087
:1055d000cb22a90000f4210001002000cc0b070021
:1055e0000080eb008080eb001e0f40005e974800bb
:1055f0001e00be00e00f5000e08f5800ebff3a00a5
:105600000080fa00000006000000fa00cbc2bf00d4
:105610000080fa00000006000200fa00000f780087
:105620001e0078006101b80000c429000012b80013
:105630006010b900050378000003430000c429008e
:105640000098b90000034300860278000400be0001
:10565000af0b07000080fa00000006000200fa000d
:10566000000f78001e0078006101b8008002200061
:105670000012b8006010b900050378000003430071
:10568000800220000098b9000003430086027800e1
:105690000400be009e0b07000080fa000000060018
:1056a0000400fa00881f78000000eb00ac0a070035
:1056b00000488800084880006140b90050f40700a5
:1056c000008fbe000800e00005003d000200200041
:1056d000037824001e00be0075f40700008fbe0092
:1056e00092282d00e3b523001e00be00f5f307004d
:1056f00082612200b3fc23006cf40700104888008c
:1057000021488800104880002148800002002000c5
:1057100003132400c3f407000000e00001003c0074
:1057200002003700caa2a9000b0037001048800011
:1057300021488000a299290093122400bbf407009d
:105740000000e0000100350002003700caa2a800f6
:1057500001003700caa2a8004f0478000080fa00b8
:10576000000006000a00fa006047980071479800a0
:10577000024f9800134f98000e8fe8001e0078002b
:105780009e489000014878001e00e8008e48900076
:10579000014878001e80e800fe4090000148780033
:1057a0009e00780063804000ee4090000148780041
:1057b0001e009000ae0090000080fa00000006007d
:1057c0000400fa00008fbe001e00be00b2fd2000e3
:1057d0009304240097f407000200200043332400c0
:1057e000b8f307000080fa00000006000400fa0089
:1057f000008fbe001e00be00b2fd200093042400f6
:10580000b0f30700020020004333240089f40700ae
:105810000080fa00000006001000fa00200798003f
:1058200031079800420798005307980064079800d2
:10583000750798004e019000de0190002e00900048
:10584000be00900077f407000000e00001003c007b
:105850001c0037006e019000fe0190002e009000a9
:10586000be00900071f407000000e0000100350068
:10587000040037002e009000be009000008fbe0094
:105880002b0037004e019000de0190006e0090006a
:10589000fe00900063f407000000e00001003c00ff
:1058a000040037006e009000fe009000008fbe00e4
:1058b0001f0037004e009000de009000008fbe00f9
:1058c0001b0037006e019000fe0190002e0090003a
:1058d000be00900053f407000000e00001003c000f
:1058e000040037002e009000be009000008fbe0024
:1058f0000f0037004e019000de0190006e00900016
:10590000fe00900049f407000000e00001003500af
:10591000040037006e009000fe009000008fbe0073
:10592000030037004e009000de009000008fbe00a4
:105930001e00be000080fa00000006000800fa0009
:105940001007980021079800320798009e009000e9
:105950002e009000808f5000110036009e009000b5
:105960003e009000808f5000030031001e00900028
:10597000000f78001a003700be0090002e00900043
:10598000808f5000030036003e009000000f78002a
:10599000130037002e009000000f78001000370031
:1059a0009e0090003e009000808f50000300360063
:1059b0001e009000000f780009003700be00900024
:1059c0002e009000808f5000030031003e009000b8
:1059d000000f7800020037002e009000000f7800c2
:1059e0001e0078000080fa00000006000c00fa009b
:1059f0001007980021079800320798004307980085
:105a0000540798009e0090002e009000808f500058
:105a1000480031009e0090003e009000808f5000b2
:105a2000440031009e0090004e009000808f500096
:105a3000400031009e0090005e009000808f50007a
:105a40003c003100de0090004e009000808f50003e
:105a50000e003600de0090003e009000808f500067
:105a60000a003600de0090002e009000808f50006b
:105a7000060036004e019000be0090002e009000ff
:105a8000aeff0700000f780049013700ce009000fc
:105a90005e009000808f50000e003600ce00900017
:105aa0003e009000808f50000a003600ce0090002b
:105ab0002e009000808f5000060036005e0190009e
:105ac000be0090002e0090009cff0700000f7800a1
:105ad00037013700be0090005e009000808f5000bc
:105ae0000e003600be0090004e009000808f5000e7
:105af0000a003600be0090002e009000808f5000fb
:105b0000060036005e019000ce0090002e0090004e
:105b10008aff0700000f7800250137005e01900022
:105b2000ce0090003e00900084ff0700000f780038
:105b30001f013700ae0090001e009000808f5000c3
:105b400048003100ae0090003e009000808f500071
:105b500044003100ae0090004e009000808f500055
:105b600040003100ae0090005e009000808f500039
:105b70003c003100de0090004e009000808f50000d
:105b80000e003600de0090003e009000808f500036
:105b90000a003600de0090001e009000808f50004a
:105ba000060036004e019000be0090001e009000de
:105bb00062ff0700000f7800fd003700ce00900064
:105bc0005e009000808f50000e003600ce009000e6
:105bd0003e009000808f50000a003600ce009000fa
:105be0001e009000808f5000060036005e0190007d
:105bf000be0090001e00900050ff0700000f7800cc
:105c0000eb003700be0090005e009000808f5000d7
:105c10000e003600be0090004e009000808f5000b5
:105c20000a003600be0090001e009000808f5000d9
:105c3000060036005e019000ce0090001e0090002d
:105c40003eff0700000f7800d90037005e0190008a
:105c5000ce0090003e00900038ff0700000f780053
:105c6000d3003700be0090001e009000808f5000cf
:105c700048003100be0090002e009000808f500040
:105c800044003100be0090004e009000808f500014
:105c900040003100be0090005e009000808f5000f8
:105ca0003c003100de0090004e009000808f5000dc
:105cb0000e003600de0090002e009000808f500015
:105cc0000a003600de0090001e009000808f500019
:105cd000060036004e019000ae0090001e009000bd
:105ce00016ff0700000f7800b1003700ce009000cb
:105cf0005e009000808f50000e003600ce009000b5
:105d00002e009000808f50000a003600ce009000d8
:105d10001e009000808f5000060036005e0190004b
:105d2000ae0090001e00900004ff0700000f7800f6
:105d30009f003700ae0090005e009000808f500002
:105d40000e003600ae0090004e009000808f500094
:105d50000a003600ae0090001e009000808f5000b8
:105d6000060036005e019000ce0090001e009000fc
:105d7000f2fe0700000f78008d0037005e019000f2
:105d8000ce0090002e009000ecfe0700000f78007f
:105d900087003700ce0090001e009000808f5000da
:105da00048003100ce0090002e009000808f5000ff
:105db00044003100ce0090003e009000808f5000e3
:105dc00040003100ce0090005e009000808f5000b7
:105dd0003c003100de0090003e009000808f5000bb
:105de0000e003600de0090002e009000808f5000e4
:105df0000a003600de0090001e009000808f5000e8
:105e0000060036003e019000ae0090001e0090009b
:105e1000cafe0700000f780065003700be00900042
:105e20005e009000808f50000e003600be00900093
:105e30002e009000808f50000a003600be009000b7
:105e40001e009000808f5000060036005e0190001a
:105e5000ae0090001e009000b8fe0700000f780012
:105e600053003700ae0090005e009000808f50001d
:105e70000e003600ae0090003e009000808f500073
:105e80000a003600ae0090001e009000808f500087
:105e9000060036005e019000be0090001e009000db
:105ea000a6fe0700000f7800410037005e01900059
:105eb000be0090002e009000a0fe0700000f7800aa
:105ec0003b003700ce0090003e009000808f5000d5
:105ed0000e003600ce0090002e009000808f500003
:105ee0000a003600ce0090001e009000808f500007
:105ef000060036003e019000ae0090001e009000ab
:105f00008efe0700000f780029003700be009000c9
:105f10004e009000808f50000e003600be009000b2
:105f20002e009000808f50000a003600be009000c6
:105f30001e009000808f5000060036004e01900039
:105f4000ae0090001e0090007cfe0700000f78005d
:105f500017003700ae0090004e009000808f500078
:105f60000e003600ae0090003e009000808f500082
:105f70000a003600ae0090001e009000808f500096
:105f8000060036004e019000be0090001e009000fa
:105f90006afe0700000f7800050037004e019000f0
:105fa000be0090002e00900064fe0700000f7800f5
:105fb0001e0078000080fa00000006000800fa00c9
:105fc00020079800310798006011b8002e0090005b
:105fd000be00900095f207000000e00001003500cf
:105fe000050037002e009000be00900001f0a200d6
:105ff000008fbe00030037002e009000be0090000e
:10600000008fbe001e00be000080fa0000000600e7
:106010000600fa00200798002e0090001007980054
:106020000e8fe8001e007800104078000080fb0012
:106030000080fa00000006000600fa002007980021
:106040002e009000100798000e8fe8001e00e80058
:10605000104078000080fb000080fa00000006007d
:106060000c00fa0010079800210798000000eb00d0
:10607000000f78002e0090000000e00003003a00be
:10608000e0ff2f00500798001c0037001000200090
:10609000300798000a0037003e009000800078002a
:1060a0001e00900000804000104078000080fb003f
:1060b0001e0f40003e0090000000e80030079800ee
:1060c000be0090002e009000808f5000f2ff39003b
:1060d000f00f20001e0f60001e00e00003003200e1
:1060e0000080eb0040079800020037000000eb0042
:1060f000400798004e009000500798005e00900006
:106100000080fa00000006000a00fa00100798005c
:1061100021079800320798000040eb00004f7800fc
:106120003e009000804178002e0090008040780072
:1061300000c8b30000c04000004178009e009000fd
:1061400000c1b3002a050700004f78001e04e000dc
:106150000500320000c8b3001e4070000000fb00c4
:10616000400798000d0037001e009000be00900010
:10617000bbff0700004f78001e04e000050032005e
:1061800000c4b3001e4070000000fb0040079800f0
:10619000020037000000eb00400798004e0090001e
:1061a0000080fa00000006001000fa00881f780046
:1061b00050079800610798000040eb00004f7800fe
:1061c0006e0090000000e000060032000e00e800c3
:1061d000820020008000eb00cbff0700004f78001a
:1061e000050037000e00e80082002000810020003a
:1061f000c5ff0700004f78001e04e00003003200d6
:106200001e00fb0070079800310037000e00e80008
:10621000204090000080fb00c800dd000e00e80078
:10622000104090000080fb0000807000cf80de00f6
:1062300073f107000200200043bb230021f1070097
:106240005e0190000089be005e0090006404400082
:106250000e00e800404090000080fb00c800dd0018
:106260000e00e800304090000080fb0000807000cd
:10627000cf80de0062f107000200200043bb230054
:1062800010f10700008cbe005e0090006804400022
:106290000e00e800604090000080fb00c800dd00b8
:1062a0000e00e800504090000080fb00008070006d
:1062b000cf80de0052f107000200200043bb230024
:1062c00000f10700008cbe000000eb007007980092
:1062d0007e0090004f0478000080fa000000060065
:1062e0000e00fa00881f7800500798000040eb006d
:1062f000004f78000e00e80082002000010120001d
:1063000081ff0700004f78001e04e0000300320008
:106310001e00fb0060079800310037000e00e80007
:10632000204090000080fb00c800dd000e00e80067
:10633000104090000080fb0000807000cf80de00e5
:106340002ff107000200200003202400b9f107000c
:106350005e0190000089be005e0090006404400071
:106360000e00e800404090000080fb00c800dd0007
:106370000e00e800304090000080fb0000807000bc
:10638000cf80de001ef10700020020000320240061
:10639000a8f10700008cbe005e0090006804400079
:1063a0000e00e800604090000080fb00c800dd00a7
:1063b0000e00e800504090000080fb00008070005c
:1063c000cf80de000ef10700020020000320240031
:1063d00098f10700008cbe000000eb0060079800f9
:1063e0006e0090004f0478000080fa000000060064
:1063f0000e00fa00881f7800500798000040eb005c
:10640000004f78000e00e80082002000810120008b
:106410003dff0700004f78001e04e000030032003b
:106420001e00fb0060079800310037000e00e800f6
:10643000204090000080fb00c800dd000e00e80056
:10644000104090000080fb0000807000cf80de00d4
:10645000ebf007000200200043cb230099f0070077
:106460005e0190000089be005e0090006404400060
:106470000e00e800404090000080fb00c800dd00f6
:106480000e00e800304090000080fb0000807000ab
:10649000cf80de00daf007000200200043cb2300ab
:1064a00088f00700008cbe005e0090006804400089
:1064b0000e00e800604090000080fb00c800dd0096
:1064c0000e00e800504090000080fb00008070004b
:1064d000cf80de00caf007000200200043cb23007b
:1064e00078f00700008cbe000000eb006007980009
:1064f0006e0090004f0478000080fa000000060053
:106500000e00fa00881f7800500798000040eb004a
:10651000004f78000e00e8008200200001022000f9
:10652000f9fe0700004f78001e04e000030032006f
:106530001e00fb0060079800310037000e00e800e5
:10654000204090000080fb00c800dd000e00e80045
:10655000104090000080fb0000807000cf80de00c3
:10656000a7f00700020020000370240031f10700ab
:106570005e0190000089be005e009000640440004f
:106580000e00e800404090000080fb00c800dd00e5
:106590000e00e800304090000080fb00008070009a
:1065a000cf80de0096f00700020020000370240078
:1065b00020f10700008cbe005e00900068044000df
:1065c0000e00e800604090000080fb00c800dd0085
:1065d0000e00e800504090000080fb00008070003a
:1065e000cf80de0086f00700020020000370240048
:1065f00010f10700008cbe000000eb00600798005f
:106600006e0090004f0478000080fa000000060041
:106610000a00fa00300798000040eb00004f7800b5
:106620000e00e8004200200081022000b6fe0700b4
:10663000004f78001e04e000030032001e00fb0043
:10664000400798000e0037000e00e8002040900040
:106650000080fb00c800dd000e00e8001040900044
:106660000080fb0000807000cf80de0064f0070037
:106670003e0190000089be000000eb00400798003a
:106680004e0090000080fa00000006000a00fa00a8
:10669000300798000040eb00004f78000e00e80043
:1066a00042002000c102200097fe0700004f780042
:1066b0001e04e000030032001e00fb0040079800ab
:1066c000110037000e00e800204090000080fb0021
:1066d000c800dd000e00e800104090000080fb00c4
:1066e00000807000cf80de0045f00700020020002f
:1066f00003482400cff007003e0190000089be004f
:106700000000eb00400798004e0090000080fa0067
:10671000000006001200fa00500798006107980078
:10672000720798000040eb00004f78000e00e80070
:10673000820020000103200073fe0700004f780054
:106740001e04e000030032001e00fb00000f980052
:106750003e0037000e00e800204090000080fb0063
:10676000c800dd000e00e800104090000080fb0033
:1067700000807000cf80de0021f0070002002000c2
:1067800003482400abf007005e0190000089be00c2
:106790000e00e800404090000080fb00c800dd00d3
:1067a0000e00e800304090000080fb000080700088
:1067b000cf80de0012f007000200200043cb230050
:1067c000c0ef07006e0190000089be000e00e800d7
:1067d000604090000080fb00c800dd000e00e80073
:1067e000504090000080fb0000807000cf80de00f1
:1067f00003f007000200200043bb2300b1ef0700b5
:10680000e4ef0700404888000e00e8006040900078
:106810000080fb00c800dd000e00e8005040900042
:106820000080fb0000807000cf80de00f4ef0700e6
:106830000200200043bb2300a2ef07007e0190006e
:106840000089be000000eb00000f98000e089000c9
:106850000080fa00000006000400fa00100798000b
:106860000000eb00000f78001e0090006100600047
:106870000004e000050032008000eb0000802000f2
:1068800049fe07000000fb001e0f70001e00900074
:106890004800de00610060000004e00005003200f6
:1068a00011002000c08020003ffe07000000fb0018
:1068b0001e0f70001e0090000000d10061006000fb
:1068c0000004e000040032008081200084fe070004
:1068d0000000fb001e0f70001e0090004200de0052
:1068e000610060000004e00004003200c08220006b
:1068f000bffe07000000fb001e0f70001e0090008e
:106900004300de00610060000004e0000600320089
:106910008280200041832000808220007dff0700cc
:106920000000fb001e0f70001e0090004400de00ff
:10693000610060000004e000040032004084200098
:10694000effe07000000fb001e0f70001e0090000d
:106950004500de00610060000004e0000400320039
:106960008082200049ff07000000fb001e0f70001e
:106970001e0090004600de00610060000004e000a0
:10698000040032000085200021ff07000000fb000a
:106990001e0f70001e0078000080fa000000060044
:1069a0000000fa000000370006c2bf00614060002e
:1069b0000004e000fcff3a0006c2bf006440600033
:1069c0000004e000f8ff3a0006c2bf006840600023
:1069d0000004e000f4ff3a0006c2bf00704060000f
:1069e0000004e000f0ff3a0009c2bf000044b2001a
:1069f0000004e000ecff3a000080fa00000006000e
:106a00000000fa0007e2a90007a2a9000782a80077
:106a10000762a9000742a9000722a8000702a900ef
:106a200006e2a90006c2a90006a2a9000682a900e2
:106a30000662a9000642a9000622a9000602a900d2
:106a4000f005200020108800c10a20009140780045
:106a5000f0c8b30000c0600001c5b3000140700081
:106a6000ace0b70008c2a9009600a90007e2a800a0
:106a700000a8210061002000a506070010002000ea
:106a80000080fa00000006000000fa0007e2a900fa
:106a90008620a9008600a9009600a900d8ff07005b
:106aa0000600070000fa20000100200098060700f9
:106ab000100020000080fa00000006000000fa002c
:106ac0008620a9009620a8000032200001002000a6
:106ad0008f060700100020000080fa00000006006a
:106ae0000000fa008620a9009620a90010002000ce
:106af0000080fa00000006000600fa0000003700df
:106b000016c2bf00614060000004e000fcff3a00d4
:106b100016c2bf00644060000004e000f8ff3a00c5
:106b200016c2bf00684060000004e000f4ff3a00b5
:106b300016c2bf00704060000004e000f0ff3a00a1
:106b400016c2bf00624060000004e000ecff3a00a3
:106b500010c0b30006e9b70008c2bf007040600073
:106b60000004e000160032000602a80000712200b6
:106b700001002000008fbe000a00370006c9bf00d8
:106b80000004e00003003a001000200020079800f5
:106b90000d0037000080eb008080eb001e0f4000ee
:106ba0005e9748001e00be00e00f5000e08f5800c6
:106bb000f2ff3a008000eb00210798000200370046
:106bc0000000eb00200798002e0090000080fa00e3
:106bd000000006000600fa0060c0b30006e9b70036
:106be00008c2bf00684060000004e00016003200e8
:106bf0000622a8000071220001002000008fbe00c4
:106c00000a00370006c9bf000004e00003003a0094
:106c100010002000200798000d0037000080eb00d6
:106c20008080eb001e0f40005e9748001e00be00f3
:106c3000e00f5000e08f5800f2ff3a008000eb00b8
:106c400021079800020037000000eb0020079800a1
:106c50002e0090000080fa00000006000200fa00fa
:106c600030c0b30006e9b70006c2bf006140600053
:106c70000004e00010003a0006c2bf00644060005b
:106c80000004e0000c003a0006c2bf00684060004b
:106c90000004e00008003a0006c2bf007040600037
:106ca0000004e00004003a0006c2bf006240600039
:106cb0000004e000030032000000eb00000f780049
:106cc0000a00370006a2a9000682a80006c9bf0074
:106cd0000004e00003003a0010002000000f7800dc
:106ce000020037000000eb00000f78001e00780063
:106cf0000080fa00000006000600fa0030c0b30071
:106d000006e9b70006c2bf00614060000004e00071
:106d100010003a0006c2bf00644060000004e000ba
:106d20000c003a0006c2bf00684060000004e000aa
:106d300008003a0006c2bf00704060000004e00096
:106d400004003a0006c2bf00624060000004e00098
:106d5000030032000000eb00200798001600370007
:106d600006a2a8000682a8000071220001002000ef
:106d7000008fbe000a00370006c9bf000004e00013
:106d800003003a0011002000210798000a00370094
:106d90000080eb008080eb001e0f40005e974800f3
:106da0001e00be00e00f5000e08f5800f2ff3a00d6
:106db0008000eb00210798002e0090000080fa0070
:106dc000000006000a00fa00300798000071220057
:106dd0000100200010079800210798000040eb00f8
:106de000004f780040c0b30006e9b70000712200f0
:106df0000100200010079800210798001d003700af
:106e000006c2bf00614060000004e00013003a00c9
:106e100006c2bf00644060000004e0000f003a00ba
:106e200006c2bf00684060000004e0000b003a00aa
:106e300006c2bf00704060000004e00007003a0096
:106e400009c2bf000044b2000004e00003003a00a1
:106e500010c0b300004f78000b0037001e009000f8
:106e6000ae00900061005000e080580010079800cc
:106e7000210798001e009000ae009000e00f500027
:106e8000e08f5800deff3a001e04e00003003a00e5
:106e90000000eb00400798001d0037000662a800c4
:106ea000006a2800110020001007980021079800b0
:106eb0001000370006c9bf000004e00007003a00d8
:106ec00000108000804078003e009000014878006b
:106ed00010002000400798000d0037001e009000b1
:106ee000ae00900061005000e0805800100798004c
:106ef000210798001e009000ae009000e00f5000a7
:106f0000e08f5800ebff3a000000eb0040079800cc
:106f10004e0090000080fa00000006000600fa0013
:106f200050c0b30006e9b7000642a8000071220075
:106f300001002000008fbe000a00370006c9bf0014
:106f40000004e00003003a00100020002007980031
:106f50000a0037000080eb008080eb001e0f40002d
:106f60005e9748001e00be00e00f5000e08f580002
:106f7000f2ff3a008000eb00210798002e009000fd
:106f80000080fa00000006000800fa004047980060
:106f900020c0b30006e9b7004e4090000000fb009f
:106fa000101088000602a8000071220001002000d5
:106fb000008fbe000a00370006c9bf000004e000d1
:106fc00003003a0010002000300798000a00370044
:106fd0000080eb008080eb001e0f40005e974800b1
:106fe0001e00be00e00f5000e08f5800f2ff3a0094
:106ff0008000eb00310798003e0090000080fa000e
:1070000000000600801f78003400f80000c0b300c4
:10701000a00188000000fa008620a9000040eb00d3
:1070200006e9b7000080fa003400f9004f0078004c
:10703000004006000200fa00000f780046f3070047
:107040000004e000fdff3a001e00780077f407001e
:1070500041f307000004e000fdff3a0037f30700aa
:107060000004e000fdff3a001e00780044f4070031
:1070700032f307000004e000fdff3a000080fa0050
:10708000000006004c04fa00889fbe008a9fbe00e4
:107090008c9fbe00e4004700001f2a000800090082
:1070a000b05878009100b1009000b100350307009e
:1070b00000482800e101200015050700040507002d
:1070c000a0030700bb030700901f2a00d9ff070099
:1070d00003040700f0202a00d6ff070089020700fa
:1070e00020222a00d3ff0700cf010700d2010700aa
:1070f00000482800e1012000050507000040eb00e2
:10710000a1ff0700ca22a800caa2a80050232a0093
:10711000c8ff070000202100a1072000fc04070091
:10712000d5c2bf00684060000004e000fcff3200f0
:107130006400470074f50700e40047000040eb00de
:1071400080489800ed004700b0012000801f7800c3
:1071500064004700801f780070242a00801f780098
:1071600001007800f2e40700e68757006d00470051
:10717000b0ff07000000eb00100798000000eb00d4
:10718000000f7800caa2a900cac2bf000080fb009d
:107190000000d100614060008040780010c0b30062
:1071a00001405000614060006140600000414000cb
:1071b000a12c200091407800d0cfb30000c0600027
:1071c00002407000cae2b7000000eb00000f780038
:1071d000b000370000482800e1012000cc0407007f
:1071e0000080eb009cfd0700404080005140800083
:1071f000824420000e0141000089be00a0418000b1
:10720000b1418000424420000e0141000089be00cf
:10721000a4428000b5428000a6428000b7428000b0
:1072200088428000994280006a4280007b42800050
:107230004c4280005d42800020428000314280004c
:10724000e24320000e0141000089be00a041800001
:10725000b1418000a24320000e0141000089be0020
:107260008041800091418000624320000e01410076
:107270000089be00604180007141800022432000ef
:107280000e0141000089be000041800011418000d4
:10729000e24220000e0141000089be00e040800073
:1072a000f1408000a24220000e0141000089be0092
:1072b000c0408000d1408000624220000e014100a9
:1072c0000089be00a0408000b14080002242200022
:1072d0000e0141000089be00804080009140800086
:1072e000e24120000e0141000089be0060408000a4
:1072f00071408000a24120000e0141000089be00c3
:107300004040800051408000624120000e01410059
:107310000089be00204080003140800022412000d2
:107320000e0141000089be00004080001140800035
:10733000e24020000e0141000089be00ed00470040
:10734000204420000e004000010878008144200005
:107350008e8040001100be00809fbe00414420008e
:107360008e8040001100be00809fbe00849fbe0042
:10737000869fbe00889fbe008a9fbe008c9fbe0075
:10738000e14320008e8040001100be00809fbe00bf
:10739000a14320008e8040001100be00809fbe00ef
:1073a000614320008e8040001100be00809fbe001f
:1073b000214320008e8040001100be00809fbe004f
:1073c000e14220008e8040001100be00809fbe0080
:1073d000a14220008e8040001100be00809fbe00b0
:1073e000614220008e8040001100be00809fbe00e0
:1073f000214220008e8040001100be00809fbe0010
:10740000e14120008e8040001100be00809fbe0040
:10741000a14120008e8040001100be00809fbe0070
:10742000614120008e8040001100be00809fbe00a0
:10743000214120008e8040001100be00809fbe00d0
:10744000e14020008e8040001100be00809fbe0001
:1074500064004700801f7800b0012000801f780082
:10746000b0012000801f7800f0252a00801f7800de
:10747000224420000e014100120078002ce4070095
:1074800080fa2f00808747006d004700e9fe070063
:107490001e0fe800f00420009e0f10004dff360084
:1074a0001e0090000000e8001007980036ff37002b
:1074b0003400f800881f780008c0b300a8018800d5
:1074c0004f0478000000fa008020a9000000fe00b0
:1074d0000080fa003400f900004006003400f80093
:1074e000881f780008c0b300a80188004f04780006
:1074f0000000fa008060a9000000fe000080fa0091
:107500003400f900004006003400f800881f7800bd
:1075100008c0b300a80188004f0478000000fa00fa
:107520008040a9000000fe000080fa003400f9004d
:10753000004006003400f800881f780008c0b3003f
:10754000a80188004f0478000000fa008080a9009c
:107550000000fe000080fa003400f9000040060040
:107560000400fa0020479800314798000040eb00e3
:10757000004f78001800370010c0b300004f7800ab
:107580005dfd07001e4f60002e4090007efe07004c
:107590001e4f60003e4090007bfe07001e4f6000c3
:1075a0008cfd07001e4f60002e4090000040e80058
:1075b00075fe07001e4f60000e00e80001fe070088
:1075c0001e4f6000ccfd070054fe07001e04e000c3
:1075d00003003a002cfd07001e04e000e6ff320025
:1075e0001e4090000000fb000080fa000000060032
:1075f0000800fa0020479800210798006247980089
:10760000734798000040eb00004f780010c0b300b3
:10761000004f780038fd07001e4f60002e4090009c
:1076200059fe07001e4f60006e40900056fe070096
:107630001e4f600067fd07001e4f60002e40900047
:107640000040e80050fe07001e4f600015003700a4
:107650002e009000dbfd07001e4f60002e00900002
:107660000000e800200798007e4090000040e900fc
:10767000704798007e4090000004e00003003a004c
:107680009dfd07001e4f60000200370073fd0700dc
:107690001e4f600006c2bf00704060000004e000a2
:1076a000fcff3a007e4090000004e000e8ff3a0052
:1076b0001afe07001e00fb000080fa000000060012
:1076c0000600fa002047980031479800424798008a
:1076d0000040eb00004f78001200370010c0b300ec
:1076e000004f780004fd07001e4f60002e40900000
:1076f00025fe07001e4f60003e40900022fe07005e
:107700001e4f60004e4090001ffe07001e4f60009d
:1077100002fe07001e4f60001e04e00003003a0056
:10772000d9fc07001e04e000ecff32001e00fb0045
:107730000080fa00000006000400fa00100798001c
:107740000040eb00004f78000040eb00104798002d
:107750001600370010c0b300004f7800e6fc0700a9
:107760001e4f600000c1b30007fe07001e4f6000ff
:1077700010c0b30004fe07001e4f600015fd070097
:107780001e4f600010c1b300fffd07001e4f6000d8
:107790000e00e8008bfd07001e4f600056fd07003d
:1077a0001e4f6000ddfd07001e4f60001e04e0005c
:1077b000e8ff32001e4090000000fb000080fa004d
:1077c000000006000600fa001007980041479800e4
:1077d0000040eb00004f78000f00370010c0b300ee
:1077e000004f7800c4fc07001e4f600000c1b300ca
:1077f000e5fd07001e4f60000040eb00e2fd0700c2
:107800001e4f600050c0b300dffd07001e4f600038
:10781000c2fd07001e4f60001e04e000efff3200b3
:107820000080fa00000006000000fa0074fc070067
:107830000080fa00000006000000fa009ffc07002c
:107840000080fa00000006000000fa00a4fc070017
:087850000080fa0000000600b0
:020000040000fa
:10785800000900000600000002000000000000000f
:1078680000000000f008000008000000020000000e
:107878000000000000000000000000006408000094
:1078880046000000020000000000000000000000a8
:1078980000000000000000000000000000000000e0
:1078a80000000000000000000000000000000000d0
:1078b80000000000000000000000000000000000c0
:1078c80000000000000000000000000000000000b0
:1078d80000000000000000000000000000000000a0
:1078e8000000000000000000f80800000800000088
:1078f800020000000000000000000000000000007e
:10790800aa08000046000000020000000000000075
:10791800000000000000000000000000000000005f
:10792800000000000000000000000000000000004f
:10793800000000000000000000000000000000003f
:10794800000000000000000000000000000000002f
:10795800000000000000000000000000000000001f
:107968000000000000000000000000000008000007
:10797800640000000000000006090000020000008a
:1079880000000000080900000200000002000000da
:1079980000000000a609000012000000020000001c
:1079a80001000200000400000800100000000000b0
:1079b800202b2d0023300000b8090000080000002b
:1079c80002000000686a6c00747a4c000000000035
:1079d8000a09000048000000020000000000000042
:1079e80000000000244000000000000000005900d2
:1079f800400000000000000088c3400000000000b4
:107a08000084d7009741000080e0370079c3410027
:107a180043176e0005b5b500b8934600f5f93f0069
:107a2800e9034f00384d32001d30f90048778200d5
:107a38005a3cbf00737fdd004f15750052090000e6
:107a480032000000020000004e414e00006e61004e
:107a58006e0049004e460000696e66000030310035
:107a680032333400353637003839610062636400d8
:107a7800656600003031320033343500363738005f
:107a88003941420043444500460000008409000093
:107a9800220000000200000030313200333435008b
:107aa800363738003961620063646500660030006b
:107ab800313233003435360037383900414243001b
:107ac8004445460000000000c00900000200000014
:107ad8000200000000000000c209000002000000cf
:107ae8000200000030000000c4090000020000008d
:0c7af80002000000000000000000000080
:020000040000fa
:107b04000000fa00410b200091407800f0c8b30057
:107b140000c0600001c6b30001407000b4e0b700cb
:107b2400901220001013880060c2a90061e2a8002e
:107b34000080fa00000006000200fa00004f7800fe
:107b440011479800e922a9001e80fb0035000700b8
:107b54001e4090000080fb0032000700e922a800cc
:107b64006022a900800720000100200067020700ae
:107b74000080fa00000006000800fa00004f7800b8
:107b840011479800224798003347980044479800cb
:107b9400554798006647980077479800e922a9005e
:107ba4001e80fb001f0007001e4090000080fb00a9
:107bb4001c0007002e4090000080fb001900070005
:107bc4003e4090000080fb00160007004e409000ed
:107bd4000080fb00130007005e4090000080fb0063
:107be400100007006e4090000080fb000d000700ad
:107bf4007e4090000080fb000a0007000ef897000a
:107c04000080fb0007000700e922a8006022a90009
:107c140080072000010020003c0207000080fa00d9
:107c2400000006000200fa00000f780063c2bf00e3
:107c3400644060000004e000030032001e0078008d
:107c44004013880003003700f00f20001e0060007e
:107c54004013880060c2bf00624060000004e0007e
:107c6400fcff3a0060c2bf00614060000004e00015
:107c7400fcff320040138000000f78000080fa00ff
:107c8400000006000600fa00004f78001107980073
:107c940042479800e922a9001e80fb00e1ff07008b
:107ca400ce4090001e00900006000700e922a800c4
:107cb4008007200001002000140207000080fa0061
:107cc400000006000400fa00000f78002147980025
:107cd400080037000c000700804078001e00780080
:107ce400014878001e0fe8002e4090000040e90093
:107cf400204798002e4090000004e000f5ff3a0071
:107d04000080fa00000006000200fa0060c2a90028
:107d14000000eb004013880060c2bf0061406000b7
:107d24000004e000fcff320060c2bf00614060005c
:107d34000004e0000d00320060c2a90063c2bf006d
:107d4400644060000004e00003003200401380003f
:107d5400000f78000700370041138000f00f200067
:107d640080806000010f7800020037000080eb0083
:107d7400000f78001e0078000080fa000000060062
:107d84000000fa00417420009140780000ceb30056
:107d940000c060003040b30044e7b70044c7bf00f0
:107da400f043b20044e7b700e0012000303a880015
:107db4000000eb00403a880040a7a90032002000f0
:107dc40081072000a0092000337420008149780035
:107dd4008049780082497800120020006104200064
:107de40070052000237420008149780080497800c0
:107df4008249780043c7bf0002c7b30082406000d5
:107e040000c3b30080cf5000faff3a0042c7bf005e
:107e14000042b2000004e000fcff32000080fa00df
:107e2400000006000000fa000000eb0020088800b3
:107e34008460a900510a200091407800f0c8b30082
:107e440000c0600001c5b30001407000a5e0b700a8
:107e54000000eb000008880000c429001008880016
:107e64000080fa00000006000000fa009460a800f8
:107e740005e1a8000080fa00000006000000fa00f6
:107e84009460a90005e1a9000080fa000000060042
:107e94000000fa000000eb00900888008500a900ab
:107ea400810a20009140780080cfb30000c06000b8
:107eb4005040b300a8e0b7000000eb005008880071
:107ec4000080fa00000006000000fa009500a800f7
:107ed40013e1a8000080fa00000006000000fa0088
:107ee4009500a90013e1a9000080fa000000060033
:107ef4000400fa00008fbe001e00be000200240031
:107f0400c3312400eee9070021ea0700d008880005
:107f140000032800f0088800110b2000914078002d
:107f2400f0c8b30000c060000044a000b1e0b70096
:107f34008760a9009760a8000080fa00000006008e
:107f44000600fa008aef0700700520002007980059
:107f5400f0fd2f0096ef070080c02c00100798005a
:107f6400d0752900000f78002e0190009e00780043
:107f74001e00900069f007000000eb002045880017
:107f84000000eb00304588000080fa000000060085
:107f94000000fa00eaff07000080fa000000060073
:107fa4000000fa00020007000080fa00000006004a
:107fb4000600fa0076ef07007005200020079800fd
:107fc400f0fd2f00afef070080602c001007980031
:107fd400d0752900000f78002e0190009e007800d3
:107fe4001e00900059f007000000eb005047880085
:107ff4000000eb00604788000080fa0000000600e3
:108004000c00fa007005200050079800700520004d
:1080140040079800f0fd2f0065ef070080c02c009a
:1080240030079800910a200091407800f0c8b3000e
:1080340000c0600001c2b30001407000a9e0b700b5
:10804400a10a20009140780080cfb30000c06000f6
:108054000014a000aae0b70080802c00300798002c
:10806400005028002007980090fb2f0085ef0700a0
:10807400310b20009140780080cfb30000c0600035
:108084003040b300b3e0b700310b200091407800da
:10809400f0c8b30000c0600001c3b3000140700029
:1080a400b3e0b70080602c0010079800d075290059
:1080b400000f78005e019000ae0090003e0090003a
:1080c40016f007004e0190009e0078001e009000fc
:1080d4001ef007000080fa00000006000000fa000d
:1080e40021e3a90021a3a9002143a8001132200003
:1080f40091407800c0cfb30000c0600021e3b70016
:10810400013220009140780000ceb30000c070001e
:1081140020e3b7002043a9002023a9002003a900dd
:1081240023c3bf007f40600023e3b7002223a900dc
:108134002203a90025e3a90025c3bf00f041b30031
:1081440025e3b700f0c3b30024e3b7000080eb00dd
:10815400501988000080fa00000006000400fa00ac
:108164001007980028e3a9001e0090007f406000db
:108174007f416000813220009140780000ceb3003e
:1081840000c060000240700028e3b7000000eb006c
:1081940070198800110020001e0090000008dd0006
:1081a400801988000080eb0050198800110020001d
:1081b4001e0090000008dd000080ea0060198800bd
:1081c40021e3a8002023a80020c3bf006140600071
:1081d4000004e000fcff320000188000000f78006b
:1081e4002023a90021e3a9001e0078000080fa00e2
:1081f4000000060087e0a900809fbe00821f78006f
:10820400f028ec00f608e20015003200f208e20063
:1082140016003200f408e200140032009147800096
:10822400420020003322af00feff3700a047800049
:108234000000e000070032000000e900f4a8b700e5
:108244003140780034e2b7000201e900f5ff3a005a
:1082540002003700f228ef00010037009147880040
:108264004f0178004f00be000040060000002000cf
:10827400b04788004f0178004f00be000040060060
:10828400f608e200feff3a0097e0a9008100e90049
:10829400a1478800b0407800a11188009047880069
:1082a40011002000b147880097e0a80000000600f4
:1082b400b0478000000006008580a900809fbe00b2
:1082c400821f7800f828ec00fe08e2001500320056
:1082d400fa08e20016003200fc08e2001400320042
:1082e400d1478000420020002322af00feff370068
:1082f400e04780000000e000070032000000e900d1
:10830400fca8b7003140780024e2b7000201e9007c
:10831400f5ff3a0002003700fa28ef0001003700a9
:10832400d14788004f0178004f00be00004006008e
:1083340000002000f04788004f0178004f00be0085
:1083440000400600fe08e200feff3a009580a90006
:108354008100e900e1478800b040780021118800dd
:10836400d047880011002000f14788009580a800bc
:1083740000000600f047800000000600809fbe0059
:108384008560a900a828ec0020458000f003b20015
:1083940041862000810040000000eb0026c2bf009f
:1083a40080487800a428ec004f00be00004006007e
:1083b4002045800031458000010050000000060087
:1083c40021458000324580000208e10008003200a7
:1083d400f203b200418620000281400092407800fe
:1083e40001487800a628ec001000200000000600d8
:1083f4000000eb0000000600809fbe0087c0a900bb
:10840400ee28ec0050478000f003b200a18a20005f
:10841400810040000000eb0036c2bf0080487800b5
:10842400ea28ec004f00be000040060050478000e0
:1084340061478000010050000000060051478000a1
:10844400624780000208e10008003200f203b20033
:10845400a18a2000028140009240780001487800ff
:10846400ec28ec0010002000000006000000eb00e7
:10847400000006000000fa00ca22a800002424001c
:10848400f100200021000700ca22a90000242400d2
:10849400f10020001d0007000080fa000000060023
:1084a4000000fa00caa2a80000242400f100200061
:1084b40016000700caa2a90000242400f10020002d
:1084c400120007000080fa00000006000000fa0015
:1084d400ca22a900c622a900caa2a900c6a2a9004c
:1084e400e4c2a900e4e2a800e502a900e522a9008b
:1084f400d302a900c602a800cb22a900c722a90062
:10850400d362a8000080fa0000000600f03fb1002a
:108514000180b10006003500ee03090000000000f0
:10852400403fb1000180b100fbff3d001000b000ee
:10853400203fb00002003500008009000000000068
:04854400000006002d
:020000040000fa
:048548000000fe0031
:00000001FF
